:0400000089EF5BF039
:08000800046ED8CF05F0E0CF33
:1000100006F00001E9CF0CF0EACF07F0E1CF08F0DD
:10002000E2CF09F0D9CF0AF0DACF0BF0F3CF12F01C
:10003000F4CF13F0FACF14F0F5CF15F0F6CF16F099
:10004000F7CF17F000C00EF001C00FF002C010F0A3
:1000500003C011F09DAA30EF00F09EBA34EF0AF011
:100060000EC000F00FC001F010C002F011C003F08C
:100070000CC0E9FF07C0EAFF078E08C0E1FF09C016
:10008000E2FF0AC0D9FF0BC0DAFF12C0F3FF13C0B2
:10009000F4FF14C0FAFF15C0F5FF16C0F6FF17C035
:1000A000F7FF045006C0E0FF05C0D8FF1000F76A54
:1000B000BE0FF66E000EF7220900F5501200000088
:1000C00000000000005F00000007000700147F141C
:1000D0007F14242A7F2A122313086462364955228A
:1000E000500005030000001C2241000041221C00BA
:1000F00014083E081408083E0808005030000008A4
:1001000008080808006060000020100804023E5142
:1001100049453E00427F40004261514946214145E8
:100120004B311814127F1027454545393C4A49493F
:100130003001710905033649494936064949291EE6
:100140000036360000005636000008142241001424
:1001500014141414004122140802015109063249F2
:1001600079413E7E1111117E7F494949363E414118
:1001700041227F4141221C7F494949417F090909A8
:10018000013E4149497A7F0808087F00417F4100CC
:100190002040413F017F081422417F404040407F82
:1001A000020C027F7F0408107F3E4141413EF76A06
:1001B000BE0FF66E010EF7220900F55012007F09FE
:1001C0000909063E4151215E7F09192946464949E0
:1001D000493101017F01013F4040403F1F20402045
:1001E0001F3F4038403F6314081463070870080736
:1001F0006151494543007F4141000204081020003D
:1002000041417F000402010204404040404000019F
:1002100002040020545454787F48444438384444FD
:100220004420384444487F3854545418087E090107
:10023000020C5252523E7F0804047800447D400074
:100240002040443D007F1028440000417F40007C56
:10025000041804787C0804047838444444387C1436
:10026000141408081414187C7C0804040848545416
:100270005420043F4440203C4040207C1C2040202F
:100280001C3C4030403C44281028440C5050503C0A
:100290004464544C44000836410000007F000000D4
:1002A0004136080010080810087846414678F76A79
:1002B000BE0FF66E020EF7220900F55012001E2145
:1002C0006121123C4140217C385456551820555527
:1002D0005578205554557820555654782054555407
:1002E000781C226222103855555518385554551827
:1002F000385455561800457C410000457D410000AA
:10030000457E4000781514157878141514787C54BF
:1003100056554424547854487E097E494938454509
:100320004538384544453838454644383C414121F4
:100330007C3C4142207C0C5150513C38454445386E
:100340003C4140413C000000000020483E49620022
:1003500000000000000000000040683E0902205438
:1003600056557800447E410038444645383C40426A
:10037000217C7C090505787C0911217C7E252526B8
:100380001800F76A920FF66E030EF7220900F55077
:100390001200FF0FFF0FFF0FFF0FFF0FFF0FFF0FE9
:1003A000FF0FFF0FFF0FFF0FFF0FFF0FFF0FFF0FDD
:1003B000FF0FFF0FFF0FFF0FFF0FFF0FFF0FFF0FCD
:1003C000FF0FFF0FFF0FFF0FFF0FFF0FFF0FFF0FBD
:1003D000FF0FFF0FFF0FFF0FFF0FFF0FFF0FFF0FAD
:1003E000FF0F0000000000000000000000000000FF
:1003F0000000F76A020FF66E040EF7220900F550AE
:100400001200FF0FFF0FFF0FFF0FFF0FFF0FFF0F78
:10041000FF0FFF0FFF0FFF0FFF0FFF0FFF0FFF0F6C
:10042000FF0F0000000000000000000000000000BE
:100430000000FF0FFF0FFF0FFF0FFF0FFF0FFF0F5A
:10044000FF0FFF0FFF0FFF0FFF0FFF0FFF0FFF0F3C
:10045000FF0F00000000000000000000000000008E
:100460000000F76A720FF66E040EF7220900F550CD
:100470001200FF0FFF0FFF0FFF0FFF0FFF0FFF0F08
:10048000FF0F0000FF0FFF0FFF0FFF0FFF0FFF0F0A
:10049000000000000000FF0FFF0FFF0FFF0F000024
:1004A0000000000000000000FF0FFF0F0000000030
:1004B000000000000000000000000000000000003C
:1004C000000000000000000000000000000000002C
:1004D0000000F76AE20FF66E040EF7220900F550ED
:1004E0001200000000000000000F000F00000000DC
:1004F000000000000000000F000F000F000F0000C0
:1005000000000000000F000F000F000F000F000F91
:10051000000000000000000F000F000F000F00009F
:100520000000000000000000000F000F00000000AD
:1005300000000000000000000000000000000000BB
:100540000000F76A520FF66E050EF7220900F5500B
:100550001200000000000000F00FF00F000000008B
:10056000000000000000F00F00000000F00F00008D
:10057000000000000000F00F00000000F00F00007D
:1005800000000000F00FF00FF00F0000F00F00006F
:100590000000F00FF00FF00FF00FF00FF00F000061
:1005A000000000000000F00F00000000F00F00004D
:1005B0000000F76AC20FF66E050EF7220900F5502B
:1005C000120000000000F00F00000000F00F00001B
:1005D000000000000000F00FF00FF00FF00FF00F20
:1005E000F00F00000000F00F0000F00FF00FF00F10
:1005F000000000000000F00F00000000F00F0000FD
:10060000000000000000F00F00000000F00F0000EC
:100610000000000000000000F00FF00F00000000DC
:100620000000F76A320FF66E060EF7220900F55049
:100630001200000000000000F00FF00F00000000AA
:10064000000000000000F00FF00FF00FF00F0000AE
:10065000000000000000F00FF00FF00FF00F00009E
:100660000000000000000000F00FF00F000000008C
:10067000000000000000F00FF00F0000000000007C
:1006800000000000F00F0000F00FF00F000000006D
:100690000000F76AA20FF66E060EF7220900F55069
:1006A0001200F00FF00FF00FF00F0000F00F00003D
:1006B00000000000F00F0000F00F0000F00FF00F3E
:1006C0000000000000000000F00F0000F00FF00F2D
:1006D0000000000000000000F00F0000000000001B
:1006E000000000000000F00FF00FF00F000000000D
:1006F0000000000000000000F00F000000000000FB
:100700000000F76A120FF66E070EF7220900F55087
:1007100012000000F76A240FF66E070EF722090098
:10072000F5501200202020202020202020202020F2
:10073000202020202000F76A460FF66E070EF722D1
:100740000900F55012002020202020202020202009
:1007500020202000F76A640FF66E070EF7220900CA
:10076000F5501200202020202020202020202020B2
:100770002020202020202020202020202020202079
:10078000202020200000F76A960FF66E070EF72251
:100790000900F5501200544954320000F76AAC0FBA
:1007A000F66E070EF7220900F5501200545045313D
:1007B0000000F76AC20FF66E070EF7220900F55027
:1007C000120054434F4E0000F76AD80FF66E070E22
:1007D000F7220900F55012005452434B0000F76A0B
:1007E000EE0FF66E070EF7220900F5501200544185
:1007F0004C420000F76A040FF66E080EF72209005B
:10080000F550120054454E430000F76A1A0FF66E79
:10081000080EF7220900F550120054594552000005
:10082000F76A300FF66E080EF7220900F550120035
:10083000434F4D4D0000F76A460FF66E080EF72243
:100840000900F5501200545858580000F76A5C0F20
:10085000F66E080EF7220900F5501200544C454E72
:100860000000F76A720FF66E080EF7220900F550C5
:1008700012004A4649460000F76A880FF66E080ED5
:10088000F7220900F5501200505249560000F76A4D
:100890009E0FF66E080EF7220900F5501200202078
:1008A0002020202020202020202020202020000088
:1008B000202A2A70617573652A2A0000202D2D30A8
:1008C00078303120254C78202D2D20007673303360
:1008D0000000202A737461727420706C7567696EF1
:1008E0002A200000202A656E6420706C7567696E8E
:1008F0002A2000000A0D206361726420696E697409
:1009000020200A0D000020636172643F3F20000038
:1009100043617264203F202020202020200061635A
:100920006D64383D257820004361726420426F6F0A
:10093000742E2E2E000073746174313D20254C7886
:10094000200073746174323D20254C78200053449C
:1009500048433D2025782000534420426F6F742E79
:100960002E2E2E2E00005344484320426F6F742ECB
:100970002E2E000073746174333D20256C782000A6
:1009800061636D6434313D2025782000202A746530
:100990006C6C206F766572666C6F772A20004D4D07
:1009A00043204D4F44452000204D4D4320426F6F62
:1009B00074000A0D20726561645F626F6F7420734A
:1009C00074617274696E67200A0D00002070726590
:1009D00020002030312000002030322000005365FC
:1009E0006356423D256C78200A0D00004270536525
:1009F000633D20256C78200A0D0053656370436CBD
:100A0000753D20256C78200A0D00525365633D200A
:100A1000256C78200A0D00004661744E3D20256C3F
:100A200078200A0D0000536563466174313D20252E
:100A30006C78200A0D00464154315F6C62615F732F
:100A4000746172743D20256C78200A0D000053708B
:100A50004661743D20256C78200A0D00524469726D
:100A6000456E744E3D20256C78200A0D000020460E
:100A7000415431362C200000536563526F6F74442B
:100A800069723D256C78200A0D006C6261526F6FAF
:100A9000744469723D256C78200A0D00456E6453DC
:100AA0006563526F6F744469723D256C78200A0D3E
:100AB00000005365637046415433323D256C782005
:100AC0000A0D0000436C75526F6F744469725F4683
:100AD000415433323D256C78200A0D005365635232
:100AE0006F6F744469723D256C78200A0D006C624A
:100AF00061526F6F744469723D256C78200A0D0055
:100B0000456E64536563526F6F744469723D256C22
:100B100078200A0D0000527372765365633D2025DC
:100B20006C78200A0D00636172645F746F74616C8D
:100B3000636C7573746572733D20256C78200A0DA3
:100B400000002121204270536563206973206E6F7D
:100B50007420353132202121200A0D002063637377
:100B6000303120002063637330322000666174737B
:100B700065637363616E3D25386C78200A0D000053
:100B800063757272656E74436C75737465723D251E
:100B9000386C78200A0D0000536563526F6F7444FF
:100BA0006972313D25386C78200A0D005365635217
:100BB0006F6F74446972313D25386C7820002A2AA1
:100BC00053656353746F703D25386C78200A0D208F
:100BD00000002A2A7365637363616E3D254C78209B
:100BE0000000726F777363616E3D254C78200000C2
:100BF000726F777363616E313D254C782000726FA0
:100C0000777363616E323D254C780A0D00004445D0
:100C10004C2000004C464E200000454E4431200040
:100C2000454E44312000454E443220004449522074
:100C30000000202D2D5C2573200A0D00202A303164
:100C40002A20000020202044656C657465204D6FCB
:100C50006465202000004400460063637330330065
:100C60004449523D2575202000006469725F6C651F
:100C700076656C3D25752020000020446972436C28
:100C800075733D25386C78200A0D00002044697288
:100C9000436C75733D25386C78200A0D00002A2AB4
:100CA0002A46494C453D20006469725F6E756D624D
:100CB00065723D25782000002020202D2D20456DD7
:100CC000707479202D2D200020202044656C6574DF
:100CD00065204D6F64652020000020202044656C55
:100CE000657465204D6F6465202000004600440057
:100CF0002046415431362C2C20006E657874436CAC
:100D000075737465723D254C78200A0D00002046ED
:100D1000415433322C2C20006E657874436C75730B
:100D20007465723D254C78200A0D0000436C757384
:100D300074657220667261676D656E746174696F47
:100D40006E203F00202D46415431362D2000202AB0
:100D5000667261673D2025782A200A0D0000202D4B
:100D600046415433322D2000202A667261673D20AF
:100D700025782A200A0D00002066696C655F6E6583
:100D800078745F636C75737465723D20256C782090
:100D90000000204641545F6C62613D20256C782044
:100DA0000000202A667261672A200000202A6E6FE8
:100DB000667261672A20000046696E64206672656B
:100DC000652046415420656E74727900202D46419D
:100DD0005431362D20002073466D3D256C78200A55
:100DE0000D000A0D2A2A20667373323D256C782087
:100DF00000007273323D256C78202A2A0A0D00000B
:100E0000206F6E6520656E64206F662066696C6574
:100E100020696E2066617431207461626C65207295
:100E2000656163686564200063633D256C78206EAE
:100E3000633D256C78200A0D0000202D4641543377
:100E4000322D200073466D3D256C78200A0D000080
:100E5000206F6E6520656E64206F662066696C6524
:100E600020696E2066617431207461626C65207245
:100E7000656163686564200063633D256C78206E5E
:100E8000633D256C78200A0D0000202A2A2A2A2A90
:100E90002047463A2046696C6520466F756E64218E
:100EA00021202A2A2A2A2A0A0D0043757272656EA9
:100EB000745F66696C656E756D6265723D25782F2D
:100EC00000006C62615F73746172743D256C782000
:100ED00000006C62615F6C656E6774683D256C78BC
:100EE000200A0D0066696C655F73746172745F63DC
:100EF0006C75737465723D256C75200A0D0066690A
:100F00006C655F73746172745F736563746F723D57
:100F1000256C75200A0D000066696C655F746F743E
:100F2000616C636C7573746572733D256C78200A0F
:100F30000D0046696C656E616D652C2053686F729B
:100F4000743D202573200A0D000046696C656E61B2
:100F50006D652C204C6F6E672028257820636861B2
:100F60007273293D202573200A0D00002A2A2A2A9F
:100F70002A2047463A2046696C65204E6F74204609
:100F80006F756E642121202A2A2A2A2A0A0D000060
:100F90002046463A202E2E2E5363616E6E696E6790
:100FA0002E2E2E2E200A0D00202A2A66696C655FDF
:100FB00073633D256C75202A200020416375727291
:100FC000656E745F66696C656E756D6265723D20F5
:100FD0002575202A200A0D00204263757272656E05
:100FE000745F66696C656E756D6265723D2025750E
:100FF000202A200A0D00202A2A7265635F73633D50
:10100000256C75202A2000000A0D20522D5C2573C6
:10101000200A0D0020522D5C2573200A0D0020426D
:1010200063757272656E745F66696C656E756D620C
:1010300065723D202575202A200A0D000A0D2A2AF6
:101040002A66696C656E616D655F73686F72743D69
:10105000202573200A0D00000A0D2A2A2A66696CD1
:10106000656E616D655F6C6F6E673D202573200A4C
:101070000D000A0D2A2A2A66696C655F6469725F31
:10108000656E7472795F6C62613D20256C75200A13
:101090000D000A0D2A2A2A4C464E5F636F756E7446
:1010A0003D202575200A0D006E65775F6469725FCB
:1010B000656E74726965735F6E65656465643D2015
:1010C0002575200A0D0066696C655F6469725F654D
:1010D0006E7472795F6C626120256C78200A0D0055
:1010E0007265635F6469725F656E7472795F6C626A
:1010F0006120256C78200A0D0000202A2A206F75B7
:1011000074206F6620726F6F7420646972202A2ABF
:101110002000456E64536563526F6F744469722A90
:1011200042705365633D20256C78200A0D0066727D
:1011300065652064697220656E74727920666F75CA
:101140006E64206174206C626120256C78200A0D29
:101150000000667265652046415420656E747279A0
:101160003D20256C78200A0D0000667265652046DA
:10117000415420656E7472795F4C4C53423D20257A
:1011800078200A0D0000667265652046415420658E
:101190006E7472795F4C4D53423D202578200A0DC4
:1011A0000000667265652046415420656E74727950
:1011B0005F4D4C53423D202578200A0D0000667299
:1011C00065652046415420656E7472795F4D4D53BC
:1011D000423D202578200A0D00004C464E5F636892
:1011E00065636B73756D5F63616C633D202578206B
:1011F0000A0D000077726974652030202A2A2A2A95
:101200002A006C62613D20256C75200A0D004F4B51
:101210002C204E65772046696C65206164646564A6
:10122000200A0D004F4B2C204E65772044697265D3
:1012300063746F7279206164646564200A0D000034
:10124000202D2D2D2D417070656E645F746F5F468B
:10125000696C652D2D2D2D2D20006C62615F6C65F4
:101260006E6774683D20256C75200A0D00006C6265
:10127000615F6D61785F6C656E6774683D20256C99
:1012800075200A0D00006C62615F6E65775F6C65AA
:101290006E6774683D20256C75200A0D0000666934
:1012A0006C655F73746172745F636C75737465727F
:1012B0003D20256C75200A0D000066696C655F7421
:1012C0006F74616C636C7573746572733D20256C0B
:1012D00075200A0D000042705365633D20256C7532
:1012E000200A0D0053656370436C753D2025752001
:1012F0002A2A200066696C655F73746172745F737B
:101300006563746F723D20256C75202A2A200000C9
:1013100066696C655F656E645F736563746F723D6B
:1013200020256C75200A0D004F4B2C206E6F20700D
:10133000726F626C656D200A0D004F4B2C206C6142
:10134000737420736563746F722062757420656EA8
:101350006F75676820737061636521200A0D000056
:10136000616464696E6720436C75737465722120D3
:101370000A0D0000204153200000667265655F631E
:101380006C75737465723D20256C75200A0D000024
:1013900066696C655F746F74616C636C757374659A
:1013A00072733D20256C75200A0D000076735F6214
:1013B00075663D20254C75200A0D0000202A6275B7
:1013C00066323D254C752000202A2A627566323D22
:1013D000254C7520000020414320000020414E2074
:1013E00000002043434120006B6270733D20254C78
:1013F00078200A0D00006B6270735F6465633D20A6
:10140000254C78200A0D000020736563735F746FAC
:10141000743D254C782000007461675F73697A65BC
:101420003D20254C78200A0D00003A003332300070
:101430003235360032323400313932003136300044
:101440003132380031313200203936002038300056
:101450002036340020353600203438002034300067
:1014600020333200202E2000036A0101BD51E50F18
:10147000E96E010E0320EA6E9EAAFED7AECFEFFF03
:10148000BDC122FD010EBD251F0BBD6FBE51BD5D4F
:1014900002E122CDBDF19E9A000130EF00F00A0D6D
:1014A0000A0D00000A0A0D20303830202D20456337
:1014B000686F4D70332076332E31202A2A207465D0
:1014C000636864657369676E2E62650A0D200000AB
:1014D00020767320696E69742073746172740A0DCA
:1014E000200020767320696E697420646F6E650A2F
:1014F0000D2000004563686F4D70332000002044CC
:10150000495920417564696F200020576176204F4A
:10151000676720576D61204D6964000020202044DA
:1015200069726563746F7269657320200000202AF8
:10153000636F756E7465644449522A2000002A2A3C
:101540002A2A2A2A2063757272656E746469723D54
:10155000202578200A0D00002A2A2A2A2A2A206318
:10156000757272656E746469723D202578200A0D6B
:1015700000002020202D2D20456D707479202D2D08
:1015800020000A0D0A0D202A2A2A2A2A7374617261
:101590007466696C653D256C75202A2A2A2A2A2AD8
:1015A0002A200A0D0000202046696C657320696EB0
:1015B000204469722E200000202A636F756E7465C6
:1015C0006446494C452A20002A2A2A2A2A2A2063CE
:1015D000757272656E7466696C653D20256C752048
:1015E0000A0D00002A2A2A2A2A2A206375727265A7
:1015F0006E7466696C653D20256C75200A0D0000CF
:101600000A0D0A0D202A2A2A322A7374617274661E
:10161000696C653D256C75202A2A2A2A2A2A2A20E7
:101620000000202A2A2A322A63757272656E746657
:10163000696C653D256C75202A2A2A2A2A2A2A20C7
:101640000000202A2A2A322A66696C655F703D25CF
:1016500075202A2A2A2A2A2A2A200000202A2A2A11
:10166000322A6469725F66696C65735B6375727256
:10167000656E746469725D3D2575202A2A2A2A2ABE
:101680002A2A200A0D0A0D000A0D555342206361D3
:10169000626C6520646973636F6E6E656374656404
:1016A0002E0A0D000A0D555342206361626C6520BD
:1016B00064657465637465642E2E2E200000696E67
:1016C000746572666163652072656164792E0000DD
:1016D000204361726420706F7765722075702E0AE6
:1016E0000D00555342204D6F646500004D4D432F52
:1016F000534420696E697420646F6E65200A0D0082
:101700004D4D432F5344207265616420626F6F74A6
:1017100020646F6E650A0D200000546F74616C20A8
:1017200046696C65733D20254C78200A0D00200A1F
:101730000D006469725F6E756D62657220254C786C
:101740003D200000746F74616C646972733D2025E4
:101750004C78200A0D006C62615F73746172743D95
:10176000254C7820000066696C655F6C62615F6C77
:10177000656E6774683D254C78200A0D0000666927
:101780006C655F746F74616C636C75737465727390
:101790002069733D20256C78200A0D0066696C6510
:1017A0005F6C62615F6C656E6774683D20256C7864
:1017B000200A0D006C6173745F6C6261733D256C6F
:1017C00078200A0D00000A0D2A2A2A202573202DD0
:1017D000202573202A2A2A0A0D20000073746172C2
:1017E0007420706C6179696E672E2E0A0D0066692F
:1017F0006C655F63757272656E745F636C7573742C
:1018000065723D25386C75200A0D000066696C65AF
:101810005F63757272656E745F736563746F723D3A
:1018200025386C75200A0D00206C62615F6375724B
:1018300072656E743D256C7820003E0020636F6DEC
:101840006D616E645F696E3D2573200A0D006C6FDB
:101850007720626174006300730072006100090008
:10186000F5520DE0F6CFDDFAF7CFDEFAF5509EA87F
:10187000FED7AD6EDDCAF6FFDECAF7FFF0D7000C6B
:10188000080EEA6E4F0EE96EEF500EE0140E016E78
:10189000006A002EFED7012EFBD7BF0E006E002E71
:1018A000FED700D0EF2EF2D7000C08015D6B8C94B0
:1018B000070E5E6F5E3D01D01FD08C945CC800F0B7
:1018C0005E51016E04E0D8900032012EFCD700B0CA
:1018D00002D08C9201D08C828C8483A00BD0010E1C
:1018E000006E5E51016E04E0D8900036012EFCD7E8
:1018F00000505D135E07DED78C945DC801F00001D7
:10190000000C0801576B566B596B586B5B6B5A6B2D
:101910008C9652C85CF80001C8DF53C85CF8C5DF7C
:1019200054C85CF8C2DF0801576B01C056F855C8AF
:101930005CF80001BADF0801596B01C058F857C8BC
:101940005BF856C85AF85AC85BF85A6B58515A2770
:1019500059515B238C865AC801F05BC802F0000124
:10196000000C0900F6CFE2FAF7CFE3FAF5509EA893
:10197000FED7AD6EE2CAF6FFE3CAF7FF0A01E12F18
:1019800001D002D00001EDD70001000C0A01E2BF36
:1019900010D00F0E006EE13900160A0E005C03E253
:1019A000300E002602D0E251002600509EA8FED73D
:1019B000AD6E0F0EE1170A0EE15D02E2300E02D0AD
:1019C000E29FE251E127E1519EA8FED7AD6E0001F2
:1019D000000C8C860A0E08014F6F000151DF8C9AB3
:1019E0000A0E08014F6F00014BDF8C8A0A0E0801B6
:1019F0004F6F000145DF83B801D0FDD7020E08010B
:101A0000526F0B0E536FFF0E546F556F000179DF4D
:101A100083B801D0FDD7020E0801526F536BCD0E73
:101A2000546F240E556F00016CDF83B801D0FDD7D1
:101A3000020E0801526F030E536F7C0E546F650E39
:101A4000556F00015EDF83B801D0FDD7020E08019B
:101A5000526F536F546B556B000153DF83B801D045
:101A6000FDD7020E0801526F0B0E536FFE0E546F1E
:101A7000556F000146DF83B801D0FDD7030E080182
:101A8000526F010E536F546B556B00013ADF02C069
:101A900044F801C043F883B801D0FDD7BC0EF66E00
:101AA000080EF76E080E0A01E16F00015ADF44C804
:101AB000E1FA570E0A01E26F000168DF43C8E1FA5C
:101AC000570E0A01E26F000161DFC70EF66E080EC5
:101AD000F76E040E0A01E16F000143DF020E0801F8
:101AE000526F010E536F200E546F480E556F000158
:101AF00008DF83B801D0FDD7020E0801526F0B0E2C
:101B0000536F37C254F837C255F80001FADE0201AC
:101B100007A506D0CC0EF66E080EF76E00019FDE0C
:101B2000020E0801526F536BCD0E546F040E556FA9
:101B30000001E7DE83B801D0FDD72EEF5CF0080E80
:101B40000A01FC6FFC530DE08A9C00D0FBBF02D061
:101B50008A9E01D08A8E00D08A8CD890FB37FC07F1
:101B6000F1D70001000C8B948B92EDCAFBFAE7DFF2
:101B70008B84000C640E08014F6F000181DE898E9A
:101B80008B848A8C8B900A0E08014F6F000178DEDF
:101B90008B80010E08014F6F000172DEAE0E0A014C
:101BA000ED6F0001E0DFA00E0A01ED6F0001DBDF49
:101BB000730E0A01ED6F0001D6DFA10E0A01ED6F71
:101BC0000001D1DF0A01ED6B0001CDDFA20E0A0199
:101BD000ED6F0001C8DF0A01ED6B0001C4DFA40E48
:101BE0000A01ED6F0001BFDFA80E0A01ED6F0001D1
:101BF000BADF3F0E0A01ED6F0001B5DFAD0E0A013D
:101C0000ED6F0001B0DF8E0E0A01ED6F0001ABDF5A
:101C1000B00E0A01ED6F0001A6DF0B0E0A01ED6F99
:101C20000001A1DFB10E0A01ED6F00019CDF310E52
:101C30000A01ED6F000197DFB30E0A01ED6F00019D
:101C400092DFF00E0A01ED6F00018DDF8A0E0A01AE
:101C5000ED6F000188DF640E0A01ED6F000183DF84
:101C60008B0E0A01ED6F00017EDF780E0A01ED6F29
:101C7000000179DF8C0E0A01ED6F000174DF640E44
:101C80000A01ED6F00016FDFBB0E0A01ED6F00016D
:101C90006ADF3E0E0A01ED6F000165DFBE0E0A012C
:101CA000ED6F000160DF3E0E0A01ED6F00015BDFAA
:101CB000870E0A01ED6F000156DF38C2EDFA53DFDF
:101CC000810E0A01ED6F00014EDF39C2EDFA4BDFE4
:101CD000820E0A01ED6F000146DF39C2EDFA43DFE3
:101CE000830E0A01ED6F00013EDF39C2EDFA3BDFE2
:101CF000AF0E0A01ED6F000136DF36EF5CF08B941A
:101D00008B82F9CAFBFA1BDFFACAFBFA18DF8B8455
:101D1000000CAE0E0A01ED6F000125DF150E0A0161
:101D2000ED6F000120DF0A01ED6B00011CDF5F0E8B
:101D30000A01ED6F000117DF750E0A01ED6F00015A
:101D400012DF0A01ED6B00010EDF3F0E0A01ED6F9D
:101D5000000109DF0801456B446B445303E1455121
:101D600018080AE00A01F96BFA6B0001C8DF0801E4
:101D7000442BD8B4452BF1D7AF0E0A01ED6F00010B
:101D8000F2DE000C150E0A01ED6F0001ECDEDECA7A
:101D9000EDFAE9DE5F0E0A01ED6F0001E4DE750E7B
:101DA0000A01ED6F0001DFDEDFCAEDFADCDE3F0E77
:101DB0000A01ED6F0001D7DE02017F6BDECA7EF201
:101DC000816BDFCA80F20001000C02017A51C70862
:101DD00003E1800E7A6FDDD07A51FC0803E1810EB9
:101DE0007A6FD7D07A51E90803E1820E7A6FD1D0A9
:101DF0007A51E20803E1830E7A6FCBD07A51E4087E
:101E000003E1840E7A6FC5D07A51E00803E1850EB4
:101E10007A6FBFD07A51E50803E1860E7A6FB9D0A8
:101E20007A51E70803E1870E7A6FB3D07A51EA0856
:101E300003E1880E7A6FADD07A51EB0803E1890E89
:101E40007A6FA7D07A51E80803E18A0E7A6FA1D0A1
:101E50007A51EF0803E18B0E7A6F9BD07A51EE082E
:101E600003E18C0E7A6F95D07A51EC0803E18D0E68
:101E70007A6F8FD07A51C40803E18E0E7A6F89D0C1
:101E80007A51C50803E18F0E7A6F83D07A51C90861
:101E900003E1900E7A6F7DD07A51E60803E1910E4E
:101EA0007A6F77D07A51C60803E1920E7A6F71D0BB
:101EB0007A51F40803E1930E7A6F6BD07A51F608E9
:101EC00003E1940E7A6F65D07A51F20803E1950E22
:101ED0007A6F5FD07A51FB0803E1960E7A6F59D082
:101EE0007A51F90803E1970E7A6F53D07A51D608E8
:101EF00003E1990E7A6F4DD07A51DC0803E19A0E16
:101F00007A6F47D07A51F80803E19B0E7A6F41D07F
:101F10007A51A30803E19C0E7A6F3BD07A51D8081E
:101F200003E19D0E7A6F35D07A51D70803E19E0EFA
:101F30007A6F2FD07A51830803E19F0E7A6F29D0F0
:101F40007A51E10803E1A00E7A6F23D07A51ED08AF
:101F500003E1A10E7A6F1DD07A51F30803E1A20EBE
:101F60007A6F17D07A51FA0803E1A30E7A6F11D075
:101F70007A51F10803E1A40E7A6F0BD07A51D1089F
:101F800003E1A50E7A6F05D07A51DF0802E1A60EB3
:101F90007A6F0001F6EF0FF00A01F435F96FF937A7
:101FA000F937F80EF917F531006E003200321F0EC6
:101FB00000160050F911F76FF539006E0036E00E8B
:101FC00000160050F611F86FF7CAF9FAF8CAFAFAD3
:101FD000000195DE000C02017A511F0802E337D19F
:101FE00006D07A517F0803E20001EFD602017A5150
:101FF000A60801E22CD17B6B7B510408D8A0D4D079
:102000007A514F080FE37A51E00F050DF3CF7CF2C0
:102010007B517C25036A000157EC00F0E8CF7DF28C
:1020200023D002017A517F080FE37A51B00F050DDA
:10203000F3CF7CF27B517C25036A0001D7EC00F0E2
:10204000E8CF7DF211D002017A51A6080DE37A5152
:10205000800F050DF3CF7CF27B517C25036A0001D4
:1020600057EC01F0E8CF7DF20A01EC6B02018651DA
:102070000A01EC5DD8B495D0EB6BEB510808D8B4ED
:102080008ED0F46B020185510F0B0A01F56FF5310B
:10209000EF6FF431EE6FEF33EE33EF33EE33EF33B8
:1020A000EE33EF33EE33EF33EE33030EEF1702016F
:1020B0008451F00B0A01F46FF56BF531F16FF431D7
:1020C000F06FF133F0333F0EF117020184510F0B23
:1020D0000A01F46FF56BF435F26FF535F36FF237F3
:1020E000F337FC0EF2177DC200F0EB51016E04E0F5
:1020F000D8900032012EFCD700A03DD0F46B020135
:1021000083510F0B0A01F56FF533F433F533F433D4
:10211000F533F433F533F433F533F433F533F43383
:10212000030EF517F425EE6F000EF521EF6F020197
:102130008251F00B0A01F46FF56BF533F433F5338C
:10214000F4333F0EF517030EF425F06F000EF52162
:10215000F16F020182510F0B0A01F46FF56BF43736
:10216000F537F437F537FC0EF417030EF425F26F4C
:10217000000EF521F36FED6B020187510A01ED5D51
:102180000BE0EECAF4FAF0CAF5FAF2CAF6FA000168
:1021900003DF0A01ED2BF0D7010EEB276ED7EC2BF6
:1021A00065D702017B2B28D70A01F46B0201855108
:1021B0000F0B0A01F56FF531EF6FF431EE6FEF336E
:1021C000EE33EF33EE33EF33EE33EF33EE33EF3303
:1021D000EE33030EEF1702018451F00B0A01F46F86
:1021E000F56BF531F16FF431F06FF133F0333F0EF1
:1021F000F117020184510F0B0A01F46FF56BF435EE
:10220000F26FF535F36FF237F337FC0EF217EC6B24
:10221000020186510A01EC5D19E0EB6BEB510808F5
:1022200013E0ED6B020187510A01ED5D0BE0EECA90
:10223000F4FAF0CAF5FAF2CAF6FA0001ADDE0A01C4
:10224000ED2BF0D7EB2BEAD7EC2BE2D70201000104
:1022500061EF11F0150E0A01ED6F000184DC7EC202
:10226000EDFA81DC02018651060DF3507E250A014C
:10227000EB6F000E02017F210A01EC6FEBCAEDFA51
:10228000000171DC750E0A01ED6F00016CDC80C28B
:10229000EDFA69DC02018751080DF35080250A012F
:1022A000EB6F000E020181210A01EC6F010EEB5F62
:1022B000000EEC5BEBCAEDFA000155DCEACA7AF2DB
:1022C0008AD602018651060DF3507E27000E7F2329
:1022D0000001000C0900F5520CE0F6CFDDFAF7CF53
:1022E000DEFAF5CFEAFAB6DFDDCAF6FFDECAF7FF9F
:1022F000F1D7000C080EEA6E450EE96EEF500EE0C5
:10230000140E016E006A002EFED7012EFBD7BF0E01
:10231000006E002EFED700D0EF2EF2D7000C080181
:102320004351080DF3CF45F80A01DE6B45C8DFFACB
:10233000000128DD0801446B4451100808E0200E1C
:102340000A01EA6F000186DF0801442BF5D700017E
:10235000000C8A88070E08014F6F4F3D01D008D04E
:102360008A94000000008A84000000004F07F5D71F
:10237000000E016E0001D9EF12F00D011F6B070E68
:10238000206F203D01D020D01ECD00F02051016EE5
:1023900004E0D8900032012EFCD700B002D08A9819
:1023A00001D08A8800008A948A8481A60BD0010E0D
:1023B000006E2051016E04E0D8900036012EFCD74B
:1023C00000501F132007DDD71FCD01F00001000CC6
:1023D000FF0E0D011E6F0001D0DF16CD1EFDCDDFFB
:1023E00018CD1CFD0D011D6B18CD1EFD0001C5DFB4
:1023F00017CD1EFDC2DF1ACD1CFD0D011D6B1ACDC0
:102400001EFD0001BADF19CD1EFDB7DF1BCD1EFD7D
:10241000B4DFFF0E0D011E6F0001AFDFFF0E0D01D7
:102420001E6F0001AADF01C090F6060190C601F000
:102430000001000C0601AC6BAB6BAA6BA96BFF0E25
:102440000D011E6F000199DF4FC81EFD96DFFF0EC4
:102450000D011E6F000191DFFF0E0D011E6F0001C7
:102460008CDFFF0E0D011E6F000187DFFF0E0D01D7
:102470001E6F000182DFFF0E0D011E6F00017DDF68
:10248000FF0E0D011E6F000178DFFF0E0D011E6FA4
:10249000000173DFFF0E0D011E6F00016EDF01C032
:1024A00050F80601AC6BAB6BAA6B50C8A9F6ABC673
:1024B000ACF6AAC6ABF6A9C6AAF6A96BFF0E0D012B
:1024C0001E6F00015ADF01C051F808015151060189
:1024D000A927000EAA23AB23AC23ABC6ACF6AAC631
:1024E000ABF6A9C6AAF6A96BFF0E0D011E6F00017F
:1024F00044DF01C052F8080152510601A927000E1D
:10250000AA23AB23AC23ABC6ACF6AAC6ABF6A9C6CE
:10251000AAF6A96BFF0E0D011E6F00012EDF01C090
:1025200053F8080153510601A927000EAA23AB2333
:10253000AC23A9C600F0AAC601F0ABC602F0ACC637
:1025400003F00001000CF40EF66E080EF76E2FEC8F
:102550000CF0899C020107A507D0060EF66E090E45
:10256000F76E00012FEC0CF00A01DE6B380EDF6F06
:10257000000108DC0201856B846B0F0E836FFF0E78
:10258000826F010E876F866F100EF66E090EF76E62
:102590000001A0DE640E08014F6F000140EC0CF05A
:1025A0008A8A4A0E0801446F443D01D005D00001DB
:1025B000D0D608014407F8D78A9A400E0D01166F4D
:1025C000186B176B1A6B196B950E1B6F000100DFF0
:1025D00001C046F8020107A50CD046C8E1FA570E23
:1025E0000A01E26F0001C6EC0CF0200E9EA8FED797
:1025F000AD6E0801462D01D007D0898CFA0E4F6FC1
:10260000000140EC0CF0A5D7480E0D01166F186BB9
:10261000176B010E1A6FAA0E196F870E1B6F000140
:10262000D7DE01C046F8020107A516D01E0EF66ED1
:10263000090EF76E060E0A01E16F0001B1EC0CF015
:1026400046C8E1FA570E0A01E26F0001C6EC0CF031
:10265000200E9EA8FED7AD6E0801462D42D0FF0E7B
:102660000D011E6F000189DE01C046F8FF0E0D014D
:102670001E6F000182DE01C046F8FF0E0D011E6FC5
:1026800000017BDE01C048F8020107A50CD048C854
:10269000E1FA570E0A01E26F0001C6EC0CF0200EC1
:1026A0009EA8FED7AD6EFF0E0D011E6F000165DE08
:1026B00001C049F8020107A50CD049C8E1FA570E3C
:1026C0000A01E26F0001C6EC0CF0200E9EA8FED7B6
:1026D000AD6E0801482D05D04951AA0802E1010E4E
:1026E000476F47530EE10A01DE6B380EDF6F0001C2
:1026F000C2EC0EF0280EF66E090EF76EEBDD1ED161
:1027000008017A0E4F6F000195DE03C04DF802C03C
:102710004CF801C04BF800C04AF8020107A52ED0C2
:10272000360EF66E090EF76E070E0A01E16F000114
:10273000B1EC0CF04DC8E1FA570E0A01E26F00014E
:10274000C6EC0CF04CC8E1FA570E0A01E26F00012A
:10275000C6EC0CF04BC8E1FA570E0A01E26F00011B
:10276000C6EC0CF04AC8E1FA570E0A01E26F00010C
:10277000C6EC0CF0200E9EA8FED7AD6E08014F6B84
:102780004BC850F84CC851F8526B4F5307E15051A9
:10279000800804E1513D02D0525301E0B2D7770ED8
:1027A0000D01166F186B176B1A6B196BFF0E1B6FF1
:1027B00000010EDE01C048F808014851FE0B02E09E
:1027C0000001C7D6690E0D01166F400E186F176B0A
:1027D0001A6B196BFF0E1B6F0001FADD01C049F87F
:1027E00008014951FE0B04E00001B3D607D00801EF
:1027F000482D03D0495301E0D2D700017A0E0801D9
:102800004F6F000117DE03C04DF802C04CF801C045
:102810004BF800C04AF8020107A52ED0420EF66E12
:10282000090EF76E070E0A01E16F0001B1EC0CF022
:102830004DC8E1FA570E0A01E26F0001C6EC0CF038
:102840004CC8E1FA570E0A01E26F0001C6EC0CF029
:102850004BC8E1FA570E0A01E26F0001C6EC0CF01A
:102860004AC8E1FA570E0A01E26F0001C6EC0CF00B
:10287000200E9EA8FED7AD6E0601FD6B08014DAD82
:1028800003D00601FD2B08014F6B4BC850F84CC814
:1028900051F8526B4F5307E15051800804E1513D0C
:1028A00002D0525306E0210E006E002EFED700012A
:1028B000A5D7020107A517D04E0EF66E090EF76ECA
:1028C000060E0A01E16F0001B1EC0CF0FDC6E1FA61
:1028D000570E0A01E26F0001C6EC0CF0200E9EA814
:1028E000FED7AD6E02010601FD5318E108014E51FD
:1028F0006408D8B002D0060111D04E2B0A01DE6B5D
:10290000380EDF6F0001C2EC0EF0580EF66E090EA5
:10291000F76EE0DC080143D710D00601FD2D0CD086
:102920000A01DE6B380EDF6F0001C2EC0EF0660E9E
:10293000F66E090EF76ECEDC080151D07A0E080152
:102940004F6F000177DD03C04DF802C04CF801C0A5
:102950004BF800C04AF8020107A52ED0740EF66E9F
:10296000090EF76E070E0A01E16F0001B1EC0CF0E1
:102970004DC8E1FA570E0A01E26F0001C6EC0CF0F7
:102980004CC8E1FA570E0A01E26F0001C6EC0CF0E8
:102990004BC8E1FA570E0A01E26F0001C6EC0CF0D9
:1029A0004AC8E1FA570E0A01E26F0001C6EC0CF0CA
:1029B000200E9EA8FED7AD6E08014F6B4BC850F895
:1029C0004CC851F8526B4F5307E15051800804E155
:1029D000513D02D0525303E00001B0D70801770EF9
:1029E0000D01166F186B176B1A6B196BFF0E1B6FAF
:1029F0000001EEDC01C046F8690E0D01166F400EB5
:102A0000186F176B1A6B196BFF0E1B6F0001E0DC60
:102A100001C046F8020107A516D0800EF66E090E19
:102A2000F76E080E0A01E16F0001B1EC0CF046C828
:102A3000E1FA570E0A01E26F0001C6EC0CF0200E1D
:102A40009EA8FED7AD6E08014651050802E118D0D8
:102A500014D0465312E0452B4551F90805E3020115
:102A600007850801BCD709D08C0EF66E090EF76EEB
:102A700000012FEC0CF0FF000801000E016E32D0B7
:102A8000020107A507D09E0EF66E090EF76E000133
:102A90002FEC0CF0FF0E0D011E6F00016EDC410EDD
:102AA0000D01166F186B176B1A6B196BFF0E1B6FEE
:102AB00000018EDC01520EE00A01DE6B380EDF6F82
:102AC0000001C2EC0EF0A80EF66E090EF76E02DCE5
:102AD0000801D6D7FF0E0D011E6F00014EDC010E5E
:102AE000016E080100015BEF3AF016CD1EFD45DCDA
:102AF00018CD1CFD0D011D6B18CD1EFD00013DDC28
:102B000017CD1EFD3ADC1ACD1CFD0D011D6B1ACD33
:102B10001EFD000132DC19CD1EFD2FDC1BCD1EFD7C
:102B20002CDCFF0E0D011E6F000127DC000C0D01D7
:102B3000156B0601FD530DE1D8900ACD0BFD09CDB3
:102B40000AFD08CD09FD0D01086B09370A370B375F
:102B5000060109CD13FD08CD12FD0ACD08FD0BCDF0
:102B600009FD0D010A6B0B6B09CD11FD08CD10FDA0
:102B70008A9AFF0E1E6F000100DC500E0D01166FC9
:102B8000186B176B020E1A6F196BFF0E1B6F00018B
:102B90001FDC015202E00D01ECD7FF0E0D011E6F8C
:102BA0000001BDEC11F0FF0E0D011E6F0001BDEC28
:102BB00011F08A8A8A9A510E0D01166F11CD18FDF7
:102BC00010CD17FD13CD1AFD12CD19FDFF0E1B6F91
:102BD00000018BDFFF0E0D011E6F0001BDEC11F037
:102BE00001C014FD0D01145303E00001F3D70D01E2
:102BF000FF0E1E6F0001BDEC11F00150FE0804E055
:102C0000010E0D011527F4D70D010F6B0E6B0F513F
:102C1000010819E30DCD03F00C510C2BD8B40D2B8A
:102C2000166F03C017FDFF0E1E6F0001BDEC11F003
:102C300017CDEAFF16CDE9FF01C0EFFF0D010E2B06
:102C4000D8B40F2BE4D7FF0E1E6F0001BDEC11F0BE
:102C50008A8A000E016E000C0A01E96BEA6B010E14
:102C6000EB6FDA6AD96A0A0EEE6FE10EED6F0A0EAB
:102C7000EA6EE50EE96EEECAE2FFEDCAE1FFEBCACD
:102C8000ECFAD890E550EE02F350E923F450EA2331
:102C9000EC2FF7D7E9CADEFFEACAE9FAEA6BD8B047
:102CA000EA2BED2BD8B4EE2BEB2BEB510508DFE133
:102CB0000001000CD8B204D00A0EEA6EF50EE96EDF
:102CC000006A016A026A036A0A01F56BF66BF76B28
:102CD000F86BF451F311F211F1112CE0200EF96FA1
:102CE000D890ED37EE37EF37F037F537F637F7375F
:102CF000F837F451F85D08E1F351F75D05E1F25161
:102D0000F65D02E1F151F55D0FE3F151F55FF2512E
:102D1000D8A0F23DF65FF351D8A0F33DF75FF45130
:102D2000D8A0F43DF85FD88000360136023603366D
:102D3000F92FD6D7F5CAEFFFF6CAECFFF7CAECFFBA
:102D4000F8CAECFF0001000CB20EF66E090EF76E29
:102D50002FEC0CF08A9AFF0E0D011E6F0001BDECE6
:102D600011F0CC0EF66E090EF76E2FEC0CF0500E33
:102D70000D01166F186B176B020E1A6F196BFF0E91
:102D80001B6F0001E8EC11F0015201E0E4D7FF0EE7
:102D90000D011E6F0001BDEC11F0FF0E0D011E6F45
:102DA0000001BDEC11F08A8AD20EF66E090EF76EA4
:102DB0002FEC0CF00D010B6B0A6B096B086B080E06
:102DC0000D6F480E0C6F0001B2DED80EF66E090EC4
:102DD000F76E2FEC0CF011CA44F80601B06BAF6B24
:102DE000AE6B44C8ADF6AFC6B0F6AEC6AFF6ADC674
:102DF000AEF6AD6B10CA45F8080145510601AD2786
:102E0000000EAE23AF23B023AFC6B0F6AEC6AFF60A
:102E1000ADC6AEF6AD6B0FCA46F8080146510601C5
:102E2000AD27000EAE23AF23B023AFC6B0F6AEC6BB
:102E3000AFF6ADC6AEF6AD6B0ECA47F80801475106
:102E40000601AD27000EAE23AF23B023020107A574
:102E500036D0DE0EF66E090EF76E060E0A01E16F31
:102E60000001B1EC0CF0B0C6E1FA570E0A01E26FB6
:102E70000001C6EC0CF0AFC6E1FA570E0A01E26F92
:102E80000001C6EC0CF0AEC6E1FA570E0A01E26F83
:102E90000001C6EC0CF0ADC6E1FA570E0A01E26F74
:102EA0000001C6EC0CF0200E9EA8FED7AD6E0A0EF7
:102EB0009EA8FED7AD6E0D0E9EA8FED7AD6EB0C615
:102EC0000BFDAFC60AFDAEC609FDADC608FD080E76
:102ED0000D010D6F480E0C6F000129DE54C844F837
:102EE0000601B86BB76BB66B44C8B5F6B7C6B8F693
:102EF000B6C6B7F6B5C6B6F6B56B53C845F8080101
:102F000045510601B527000EB623B723B8230201A9
:102F100007A536D0EC0EF66E090EF76E070E0A0105
:102F2000E16F0001B1EC0CF0B8C6E1FA570E0A01EE
:102F3000E26F0001C6EC0CF0B7C6E1FA570E0A01C9
:102F4000E26F0001C6EC0CF0B6C6E1FA570E0A01BA
:102F5000E26F0001C6EC0CF0B5C6E1FA570E0A01AB
:102F6000E26F0001C6EC0CF0200E9EA8FED7AD6EFD
:102F70000A0E9EA8FED7AD6E0D0E9EA8FED7AD6EB2
:102F80000601946B936B926B55C891F6020107A5ED
:102F900037D0FA0EF66E090EF76E090E0A01E16FD0
:102FA0000001B1EC0CF094C6E1FA570E0A01E26F91
:102FB0000001C6EC0CF093C6E1FA570E0A01E26F6D
:102FC0000001C6EC0CF092C6E1FA570E0A01E26F5E
:102FD0000001C6EC0CF091C6E1FA570E0A01E26F4F
:102FE0000001C6EC0CF0200E9EA8FED7AD6E0A0EB6
:102FF0009EA8FED7AD6E0D0E9EA8FED7AD6E020147
:1030000057C844F80601A06B9F6B9E6B44C89DF6A1
:103010009FC6A0F69EC69FF69DC69EF69D6B56C89F
:1030200045F80801455106019D27000E9E239F2368
:10303000A023020107A536D00A0EF66E0A0EF76E1F
:10304000060E0A01E16F0001B1EC0CF0A0C6E1FA36
:10305000570E0A01E26F0001C6EC0CF09FC6E1FAC0
:10306000570E0A01E26F0001C6EC0CF09EC6E1FAB1
:10307000570E0A01E26F0001C6EC0CF09DC6E1FAA2
:10308000570E0A01E26F0001C6EC0CF0200E9EA85C
:10309000FED7AD6E0A0E9EA8FED7AD6E0D0E9EA891
:1030A000FED7AD6E0601986B976B966B58C895F678
:1030B000020107A536D0180EF66E0A0EF76E060E40
:1030C0000A01E16F0001B1EC0CF098C6E1FA570E6D
:1030D0000A01E26F0001C6EC0CF097C6E1FA570E48
:1030E0000A01E26F0001C6EC0CF096C6E1FA570E39
:1030F0000A01E26F0001C6EC0CF095C6E1FA570E2A
:103100000A01E26F0001C6EC0CF0200E9EA8FED76B
:10311000AD6E0A0E9EA8FED7AD6E0D0E9EA8FED710
:10312000AD6E06019D51AD25B16F9E51AE21B26FBE
:103130009F51AF21B36FA051B021B46F020107A519
:1031400036D0260EF66E0A0EF76E090E0A01E16FF2
:103150000001B1EC0CF0B4C6E1FA570E0A01E26FBF
:103160000001C6EC0CF0B3C6E1FA570E0A01E26F9B
:103170000001C6EC0CF0B2C6E1FA570E0A01E26F8C
:103180000001C6EC0CF0B1C6E1FA570E0A01E26F7D
:103190000001C6EC0CF0200E9EA8FED7AD6E0A0E04
:1031A0009EA8FED7AD6E0D0E9EA8FED7AD6EB4C61E
:1031B000E4FAB3C6E3FAB2C6E2FAB1C6E1FAB8C6B7
:1031C000E8FAB7C6E7FAB6C6E6FAB5C6E5FA000108
:1031D00043DD03C0C4F602C0C3F601C0C2F600C09E
:1031E000C1F6020107A537D0360EF66E0A0EF76E4D
:1031F000100E0A01E16F0001B1EC0CF0C4C6E1FA57
:10320000570E0A01E26F0001C6EC0CF0C3C6E1FAEA
:10321000570E0A01E26F0001C6EC0CF0C2C6E1FADB
:10322000570E0A01E26F0001C6EC0CF0C1C6E1FACC
:10323000570E0A01E26F0001C6EC0CF0200E9EA8AA
:10324000FED7AD6E0A0E9EA8FED7AD6E0D0E9EA8DF
:10325000FED7AD6E02015FC844F80601A46BA36BF4
:10326000A26B44C8A1F6A3C6A4F6A2C6A3F6A1C643
:10327000A2F6A16B5EC845F8080145510601A127D9
:10328000000EA223A323A4234E0EF66E0A0EF76EA1
:10329000070E0A01E16F0001B1EC0CF0A4C6E1FADF
:1032A000570E0A01E26F0001C6EC0CF0A3C6E1FA6A
:1032B000570E0A01E26F0001C6EC0CF0A2C6E1FA5B
:1032C000570E0A01E26F0001C6EC0CF0A1C6E1FA4C
:1032D000570E0A01E26F0001C6EC0CF0200E9EA80A
:1032E000FED7AD6E0A0E9EA8FED7AD6E0D0E9EA83F
:1032F000FED7AD6E5AC844F80601A86BA76BA66B43
:1033000044C8A5F6A7C6A8F6A6C6A7F6A5C6A6F6FB
:10331000A56B59C845F8080145510601A527000EBF
:10332000A623A723A823020107A536D05C0EF66EBC
:103330000A0EF76E0A0E0A01E16F0001B1EC0CF003
:10334000A8C6E1FA570E0A01E26F0001C6EC0CF0C4
:10335000A7C6E1FA570E0A01E26F0001C6EC0CF0B5
:10336000A6C6E1FA570E0A01E26F0001C6EC0CF0A6
:10337000A5C6E1FA570E0A01E26F0001C6EC0CF097
:10338000200E9EA8FED7AD6E0A0E9EA8FED7AD6E8B
:103390000D0E9EA8FED7AD6E94C6E4FA93C6E3FA6E
:1033A00092C6E2FA91C6E1FAB8C6E8FAB7C6E7FAF9
:1033B000B6C6E6FAB5C6E5FA00014EDC03C0C8F6AB
:1033C00002C0C7F601C0C6F600C0C5F60601A55387
:1033D00007E1A65305E1A75303E1A853D8B468D188
:1033E000A15307E1A25305E1A35303E1A453D8B4C9
:1033F0005FD16E0EF66E0A0EF76E00012FEC0CF028
:1034000002013197A4C6E4FAA3C6E3FAA2C6E2FA1F
:10341000A1C6E1FA98C6E8FA97C6E7FA96C6E6FAB0
:1034200095C6E5FA000118DC00500601B125D16F00
:103430000150B221D26F0250B321D36F0350B42197
:10344000D46F020107A536D0780EF66E0A0EF76E1D
:103450000B0E0A01E16F0001B1EC0CF0D4C6E1FAE9
:10346000570E0A01E26F0001C6EC0CF0D3C6E1FA78
:10347000570E0A01E26F0001C6EC0CF0D2C6E1FA69
:10348000570E0A01E26F0001C6EC0CF0D1C6E1FA5A
:10349000570E0A01E26F0001C6EC0CF0200E9EA848
:1034A000FED7AD6E0A0E9EA8FED7AD6E0D0E9EA87D
:1034B000FED7AD6ED4C6E4FAD3C6E3FAD2C6E2FABA
:1034C000D1C6E1FAB8C6E8FAB7C6E7FAB6C6E6FA70
:1034D000B5C6E5FA00012CEC16F003C0DCF602C01C
:1034E000DBF601C0DAF600C0D9F6020107A536D036
:1034F0008A0EF66E0A0EF76E0B0E0A01E16F0001DE
:10350000B1EC0CF0DCC6E1FA570E0A01E26F0001E3
:10351000C6EC0CF0DBC6E1FA570E0A01E26F0001BF
:10352000C6EC0CF0DAC6E1FA570E0A01E26F0001B0
:10353000C6EC0CF0D9C6E1FA570E0A01E26F0001A1
:10354000C6EC0CF0200E9EA8FED7AD6E0A0E9EA80B
:10355000FED7AD6E0D0E9EA8FED7AD6E0601A53549
:103560000A01486F0601A6350A01496F0601A73511
:103570000A014A6F0601A8350A014B6F48374937DF
:103580004A374B37483749374A374B374837493737
:103590004A374B37483749374A374B37E00E4817D9
:1035A000D8924BCAF0FA4ACAEFFA49CAEEFA48CAA8
:1035B000EDFAB8C6F4FAB7C6F3FAB6C6F2FAB5C66B
:1035C000F1FA00015AEC16F000500601D125D56F32
:1035D0000150D221D66F0250D321D76F0350D4218E
:1035E000D86F020107A536D09C0EF66E0A0EF76E54
:1035F0000E0E0A01E16F0001B1EC0CF0D8C6E1FA41
:10360000570E0A01E26F0001C6EC0CF0D7C6E1FAD2
:10361000570E0A01E26F0001C6EC0CF0D6C6E1FAC3
:10362000570E0A01E26F0001C6EC0CF0D5C6E1FAB4
:10363000570E0A01E26F0001C6EC0CF0200E9EA8A6
:10364000FED7AD6E0A0E9EA8FED7AD6E0D0E9EA8DB
:10365000FED7AD6EA3C64BFAA2C64AFAA1C649FA76
:103660000A01486B06019D510A01485F06019E51FF
:103670000A01495B06019F510A014A5B0601A051FC
:103680000A014B5B0601AD510A01485D0601C96F95
:10369000AE510A0149590601CA6FAF510A014A5990
:1036A0000601CB6FB0510A014B590601CC6F31D2E4
:1036B000020131876FC844F80601BC6BBB6BBA6B63
:1036C00044C8B9F6BBC6BCF6BAC6BBF6B9C6BAF6AC
:1036D000B96B6EC845F8080145510601B927000EBF
:1036E000BA23BB23BC23BBC6BCF6BAC6BBF6B9C65D
:1036F000BAF6B96B6DC846F8080146510601B927FC
:10370000000EBA23BB23BC23BBC6BCF6BAC6BBF6AD
:10371000B9C6BAF6B96B6CC847F80801475106013B
:10372000B927000EBA23BB23BC23020107A537D05B
:10373000B20EF66E0A0EF76E0A0E0A01E16F000174
:10374000B1EC0CF0BCC6E1FA570E0A01E26F0001C1
:10375000C6EC0CF0BBC6E1FA570E0A01E26F00019D
:10376000C6EC0CF0BAC6E1FA570E0A01E26F00018E
:10377000C6EC0CF0B9C6E1FA570E0A01E26F00017F
:10378000C6EC0CF0200E9EA8FED7AD6E0A0E9EA8C9
:10379000FED7AD6E0D0E9EA8FED7AD6E020177C8A6
:1037A00044F80601C06BBF6BBE6B44C8BDF6BFC614
:1037B000C0F6BEC6BFF6BDC6BEF6BD6B76C845F840
:1037C000080145510601BD27000EBE23BF23C023BB
:1037D000BFC6C0F6BEC6BFF6BDC6BEF6BD6B75C8D9
:1037E00046F8080146510601BD27000EBE23BF233F
:1037F000C023BFC6C0F6BEC6BFF6BDC6BEF6BD6B13
:1038000074C847F8080147510601BD27000EBE23C2
:10381000BF23C023020107A536D0C40EF66E0A0EE0
:10382000F76E110E0A01E16F0001B1EC0CF0C0C699
:10383000E1FA570E0A01E26F0001C6EC0CF0BFC6B8
:10384000E1FA570E0A01E26F0001C6EC0CF0BEC6A9
:10385000E1FA570E0A01E26F0001C6EC0CF0BDC69A
:10386000E1FA570E0A01E26F0001C6EC0CF0200EDF
:103870009EA8FED7AD6E0A0E9EA8FED7AD6E0D0EA9
:103880009EA8FED7AD6EBCC6E4FABBC6E3FABAC6C4
:10389000E2FAB9C6E1FA98C6E8FA97C6E7FA96C618
:1038A000E6FA95C6E5FA00012CEC16F003C0D4F652
:1038B00002C0D3F601C0D2F600C0D1F60601B15164
:1038C000D127B251D223B351D323B451D42302010F
:1038D00007A536D0DC0EF66E0A0EF76E0B0E0A0147
:1038E000E16F0001B1EC0CF0D4C6E1FA570E0A0109
:1038F000E26F0001C6EC0CF0D3C6E1FA570E0A01E4
:10390000E26F0001C6EC0CF0D2C6E1FA570E0A01D4
:10391000E26F0001C6EC0CF0D1C6E1FA570E0A01C5
:10392000E26F0001C6EC0CF0200E9EA8FED7AD6E33
:103930000A0E9EA8FED7AD6E0D0E9EA8FED7AD6EE8
:10394000D4C6E4FAD3C6E3FAD2C6E2FAD1C6E1FAA3
:10395000B8C6E8FAB7C6E7FAB6C6E6FAB5C6E5FAF3
:1039600000012CEC16F003C0DCF602C0DBF601C04F
:10397000DAF600C0D9F6020107A536D0EE0EF66ED3
:103980000A0EF76E0B0E0A01E16F0001B1EC0CF0AC
:10399000DCC6E1FA570E0A01E26F0001C6EC0CF03A
:1039A000DBC6E1FA570E0A01E26F0001C6EC0CF02B
:1039B000DAC6E1FA570E0A01E26F0001C6EC0CF01C
:1039C000D9C6E1FA570E0A01E26F0001C6EC0CF00D
:1039D000200E9EA8FED7AD6E0A0E9EA8FED7AD6E35
:1039E0000D0E9EA8FED7AD6E06019151D125D56F63
:1039F0009251D221D66F9351D321D76F9451D421B4
:103A0000D86F020107A536D0000EF66E0B0EF76ECA
:103A10000E0E0A01E16F0001B1EC0CF0D8C6E1FA1C
:103A2000570E0A01E26F0001C6EC0CF0D7C6E1FAAE
:103A3000570E0A01E26F0001C6EC0CF0D6C6E1FA9F
:103A4000570E0A01E26F0001C6EC0CF0D5C6E1FA90
:103A5000570E0A01E26F0001C6EC0CF0200E9EA882
:103A6000FED7AD6E0A0E9EA8FED7AD6E0D0E9EA8B7
:103A7000FED7AD6E0601B9350A01486F0601BA35A9
:103A80000A01496F0601BB350A014A6F0601BC35C0
:103A90000A014B6F483749374A374B374837493760
:103AA0004A374B37483749374A374B374837493712
:103AB0004A374B37483749374A374B374837493702
:103AC0004A374B37800E481706019D510A01485F5F
:103AD00006019E510A01495B06019F510A014A5B9A
:103AE0000601A0510A014B5B0601AD510A01485D78
:103AF0000601C96FAE510A0149590601CA6FAF519B
:103B00000A014A590601CB6FB0510A014B5906010F
:103B1000CC6F020107AB37D0160EF66E0B0EF76EA8
:103B2000090E0A01E16F0001B1EC0CF0A0C6E1FA48
:103B3000570E0A01E26F0001C6EC0CF09FC6E1FAD5
:103B4000570E0A01E26F0001C6EC0CF09EC6E1FAC6
:103B5000570E0A01E26F0001C6EC0CF09DC6E1FAB7
:103B6000570E0A01E26F0001C6EC0CF0200E9EA871
:103B7000FED7AD6E0A0E9EA8FED7AD6E0D0E9EA8A6
:103B8000FED7AD6E020107AB37D0260EF66E0B0ED8
:103B9000F76E140E0A01E16F0001B1EC0CF0CCC617
:103BA000E1FA570E0A01E26F0001C6EC0CF0CBC639
:103BB000E1FA570E0A01E26F0001C6EC0CF0CAC62A
:103BC000E1FA570E0A01E26F0001C6EC0CF0C9C61B
:103BD000E1FA570E0A01E26F0001C6EC0CF0200E6C
:103BE0009EA8FED7AD6E0A0E9EA8FED7AD6E0D0E36
:103BF0009EA8FED7AD6E0201D4C6D0F6D3C6CFF6CE
:103C0000D2C6CEF6D1C6CDF60601B55307E1B65100
:103C1000020804E1B75302E1B85309E0420EF66E20
:103C20000B0EF76E00012FEC0CF0FF0006010001F7
:103C300068EF3AF00A01E7CAEDFAE8CAEEFAE9CA13
:103C4000E7FAEACAE8FAE96BEA6BE7CAEBFAE8CA0C
:103C5000ECFA8A9AFF0E0D011E6F0001BDEC11F007
:103C6000500E0D01166F186B176B1A6B010E196F42
:103C7000FF0E1B6F0001E8EC11F0015202E00A0197
:103C8000E9D7FF0E0D011E6F0001BDEC11F0FF0E14
:103C90000D011E6F0001BDEC11F08A8A8A9A510E47
:103CA0000D01166FECCA18FDEBCA17FDEECA1AFD1E
:103CB000EDCA19FDFF0E1B6F000175EC15F0FF0E2C
:103CC0000D011E6F0001BDEC11F001C0F0FA0A01F8
:103CD000F05302E00001F3D7FF0E0D011E6F00014B
:103CE000BDEC11F00150FE0802E00A01F5D7FF0E0D
:103CF0000D011E6F0001BDEC11F001C0EFFAFF0EC7
:103D00000D011E6F0001BDEC11F08A8AEFCA00F0B0
:103D1000016A026A036A000CEACAFAFAE9CAF9FA05
:103D2000E8CAF8FAE7CAF7FAEACAF2FAE9CAF1FA0F
:103D3000E8CAF0FAE7CAEFFAD8900A01FA31FE6F42
:103D4000F931FD6FF831FC6FD890EF6BFC35F06FF7
:103D5000FD35F16FFE35F26FD890EE6BF231ED6FFD
:103D6000F131EC6FF031EB6FEF51F75DF36FF05124
:103D7000F859F46FF151F959F56FF251FA59F66F9C
:103D8000EB510601885D0FE10A01EC510601895DE6
:103D90000AE10A01ED5106018A5D05E10A01EE51D1
:103DA00006018B5D18E0EECA0BFDEDCA0AFDECCAF8
:103DB00009FDEBCA08FD040E0D010D6F880E0C6F96
:103DC000000197EC15F0EECA8BF6EDCA8AF6ECCA44
:103DD00089F6EBCA88F6880E0A01F325E96E040E0F
:103DE000F421EA6EEFCFFBFAFBCA01F00001000CF0
:103DF000EACAEEFAE9CAEDFAEECA03F00A01EDCA20
:103E0000E9FFEECAEAFFEF522AE0ECCAF0FAEBCA89
:103E1000EFFAF0CA03F0EFCAE9FFF0CAEAFFEF5287
:103E200018E0EDCAE9FFEECAEAFFEFCFF1FAF0CAF7
:103E300003F0EFCAE9FFF0CAEAFFEF50F15D05E1D8
:103E4000EDCA01F0EECA02F00DD0EF2BD8B4F02B82
:103E5000E0D7ED2BD8B4EE2B0001CED70A01000E2F
:103E6000016E026E000147EF1FF0200E0A01E36FA2
:103E7000E46BE2CAE8FAE1CAE7FAE2CAEAFAE1CA9E
:103E8000E9FA0A0EEC6FE30EEB6F0001B1D702C046
:103E9000E6FA01C0E5FA0A01E151E55D07E1E25108
:103EA000E65D04E1E12BD8B4E22B64D0E55341E1B7
:103EB000E6533FE1E2CA03F0E1CAE9FFE2CAEAFFE2
:103EC000EF521BE0E8CA03F0E751E72BD8B4E82B28
:103ED000E96F03C0EAFAE2CA03F0E151E12BD8B47A
:103EE000E22BE96E03C0EAFFEFCFEBFAEACAEAFF82
:103EF000E9CAE9FFEBCAEFFFDDD7E751D8B4E8071D
:103F0000E707E8CA03F0E7CAE9FFE8CAEAFFEF50AB
:103F1000200806E1E7CAE9FFE8CAEAFFEF6A08D02D
:103F2000E72BD8B4E82BE7CAE9FFE8CAEAFFEF6A53
:103F300021D0E151E55D03E1E251E65D1BE0E8CA15
:103F400003F0E751E72BD8B4E82BE96F03C0EAFA96
:103F5000E2CA03F0E151E12BD8B4E22BE96E03C0D1
:103F6000EAFFEFCFEBFAEACAEAFFE9CAE9FFEBCAD8
:103F7000EFFFDFD7E55381E1E653D8A47ED7E8CA47
:103F8000E2FAE7CAE1FA000138EF23F0E2CAE4FA04
:103F9000E1CAE3FAE4CA03F00A01E3CAE9FFE4CAAA
:103FA000EAFFEF5206E0E32BD8B4E42B0001F2D78E
:103FB0000A01E151E35D006EE251E459036E00C075
:103FC00001F00001000CE2CAE8FAE1CAE7FA0A01CE
:103FD000E55302E1E65327E0E4CA03F0E3CAE9FF50
:103FE000E4CAEAFFEF521FE0E8CA03F0E751E72B0B
:103FF000D8B4E82BE96F03C0EAFAE4CA03F0E3514E
:10400000E32BD8B4E42BE96E03C0EAFFEFCFEBFA61
:10401000EACAEAFFE9CAE9FFEBCAEFFFE551D8B403
:10402000E607E507D5D7E55302E1E6530FE0E8CA16
:1040300003F0E751E72BD8B4E82BE96E03C0EAFFA1
:10404000EF6AE551D8B4E607E507EDD7E1CA01F01C
:10405000E2CA02F00001000CEF5210E0EACFE2FAEF
:10406000E9CFE1FAEF509EA8FED7AD6EE2CAEAFFB3
:10407000E1CAE9FFE92AD8B4EA2AEED7000CE950F0
:104080000A01E56F3B0EEC6F9A0EEB6FCA0EEA6FFA
:10409000E96B0A0EE76FD8820A0EEA6EE10EE96E4E
:1040A000E4CAF0FAE3CAEFFAE2CAEEFAE1CAEDFABC
:1040B000ECCAF4FAEBCAF3FAEACAF2FAE9CAF1FA7C
:1040C00000015AEC16F00150005213E10A01E751C9
:1040D000010AD8A402D000010CD0E5510CE00F0B6E
:1040E000E75D01E00EE2E5BF0CD0E5BD04D0200E97
:1040F00003D00A01E56B300E002600509EA8FED7C3
:10410000AD6ED892ECCAF0FAEBCAEFFAEACAEEFA50
:10411000E9CAEDFAF46BF36BF26B0A0EF16F000172
:104120005AEC16F003C0ECFA02C0EBFA01C0EAFA4E
:1041300000C0E9FA0A01E72FAED70001000C0A011E
:10414000E451016AE35D03E2E3CA00F00CD0006AC7
:10415000080EE56FE3370036E451005CD8B0006E1E
:104160000136E52FF7D70001000C0150E1CAE3FA50
:10417000640E0A01E46F0001E2DF00C0E1FA0150C1
:10418000300E08E10A01E2A30ED0E2B70CD0E2B98A
:10419000200E04D00A01E297E299E2810126015043
:1041A0009EA8FED7AD6EE1CAE3FA0A0EE46F0001E5
:1041B000C6DF00C0E1FA0150300E08E10A01E2B7A3
:1041C0000BD0E2A109D0E2B9200E00010126015076
:1041D0009EA8FED7AD6E0A01300EE127E1519EA8E0
:1041E000FED7AD6E0001000CE8CAFDFCE7CAFCFC7E
:1041F000E6CAFBFCE5CAFAFCE8CAF5FCE7CAF4FC2F
:10420000E6CAF3FCE5CAF2FCD8900C01FD310D01C1
:104210000A6F0C01FC310D01096F0C01FB310D011E
:10422000086FD8900C01F26B0D0108350C01F36F8B
:104230000D0109350C01F46F0D010A350C01F56F04
:10424000D890EE6BF531ED6FF431EC6FF331EB6F2D
:10425000F251FA5DF66FF351FB59F76FF451FC59C7
:10426000F86FF551FD59F96F0A01EA5302E0EA2DA2
:1042700010D0EECC0BFDEDCC0AFDECCC09FDEBCC67
:1042800008FD0A0E0D010D6FEB0E0C6F000197EC8F
:1042900015F0EB0E0C01F625E96E0A0EF721EA6E19
:1042A000E9CAEFFF0A01EA2D01D003D0EA51020862
:1042B00003E1000E016EC9D08A9A500E0D01166FEF
:1042C000186B176B020E1A6F196B010E1B6F000132
:1042D000E8EC11F001C0EFFC0C01EF5302E00A0121
:1042E000EBD7FF0E0D011E6F0001BDEC11F0FF0EAC
:1042F0000D011E6F0001BDEC11F08A8A8A9A060139
:10430000FD532AE1F2CC02FD0C01F3CC03FD0D01BB
:10431000F4CCF2FCF5CCF3FC0C01F46BF56BF2CCB5
:1043200000FD0C01F3CC01FD0D01FF0E1E6F00011D
:10433000BDEC11F0580E0D01166F01CD18FD00CD2A
:1043400017FD03CD1AFD02CD19FD010E1B6F0001F3
:1043500075EC15F02BD00601FD2D28D0EBCC06FD19
:104360000C01ECCC07FD0D01EDCCEBFCEECCECFC34
:104370000C01ED6BEE6BEBCC04FD0C01ECCC05FD00
:104380000D01FF0E1E6F0001BDEC11F0580E0D0166
:10439000166F05CD18FD04CD17FD07CD1AFD06CD0E
:1043A00019FD010E1B6F000175EC15F0FF0E0D01DC
:1043B0001E6F0001BDEC11F001C0EFFC0C01EF53CA
:1043C00002E000019BD7FE0E0D011E6F0001BDEC47
:1043D00011F00C01F16BF06BF05303E1F1510208A5
:1043E00012E0EB0EF025E96E0A0EF121EA6EEFCF36
:1043F00008FD08CD1EFD0001BDEC11F00C01F02BF5
:10440000D8B4F12BE9D7FF0E0D011E6F0001BDECF2
:1044100011F001C0EFFC0C01EF511F0B050801E08A
:10442000F2D7FF0E0D011E6F0001BDEC11F001C0AF
:10443000EFFC0C01EF3D01D005D0FE2BD8B4FF2BD3
:10444000F0D7F8D7000E016E0A010001000C070E2C
:10445000EA6E660EE96E000E9BEC03F00A0009009E
:10446000F550EE6E0009FBE10701666B0601FD5396
:1044700038E10A01DD6BDD51080831E0036ADD51E6
:10448000660F016E070E032201C0E1FA03C0E2FAD3
:10449000DD5107015C250A01E36F000E07015D2174
:1044A0000A01E46F000E07015E210A01E56F000EAC
:1044B00007015F210A01E66FEA6FE5CAE9FAE4CA7B
:1044C000E8FAE3CAE7FA00011AEC1EF0E2CAEAFFD2
:1044D000E1CAE9FF00C0EFFF0A01DD2BCCD739D0DC
:1044E0000601FD2D37D00A01DD6BDD51080831E0F2
:1044F000036ADD51660F016E070E032201C0E1FA67
:1045000003C0E2FADD5107015C250A01E36F000EEA
:1045100007015D210A01E46F000E07015E210A0117
:10452000E56F000E07015F210A01E66FEA6FE5CA39
:10453000E9FAE4CAE8FAE3CAE7FA00018CEC1EF0F3
:10454000E2CAEAFFE1CAE9FF01C0EFFF0A01DD2B81
:10455000CCD70601FD5340E1090E0A01DD6FDD51A4
:104560000C0838E0036ADD51660F016E070E032266
:1045700001C0E1FA03C0E2FADD5107015C250A013E
:10458000E36F000E07015D210A01E46F000E0701D1
:104590005E210A01E56F000E07015F210A01E66F47
:1045A000010EE35F000EE45BE55BE65BE6CAEAFA58
:1045B000E5CAE9FAE4CAE8FAE3CAE7FA00011AEC44
:1045C0001EF0E2CAEAFFE1CAE9FF00C0EFFF0A01FC
:1045D000DD2BC5D741D00601FD2D3ED0090E0A01C5
:1045E000DD6FDD510C0838E0036ADD51660F016EA6
:1045F000070E032201C0E1FA03C0E2FADD51070110
:104600005C250A01E36F000E07015D210A01E46FDA
:10461000000E07015E210A01E56F000E07015F2110
:104620000A01E66F010EE35F000EE45BE55BE65B0B
:10463000E6CAEAFAE5CAE9FAE4CAE8FAE3CAE7FA36
:1046400000018CEC1EF0E2CAEAFFE1CAE9FF01C0FA
:10465000EFFF0A01DD2BC5D72E0E07016E6F736BBE
:10466000070E0A01E26F660EE16F000135EF1FF0E1
:10467000070EEA6E750EE96E000EAAEC03F00A0052
:104680000900F550EE6E0009FBE10701756BAE6B9A
:10469000606B0601FD53D8A415D2050E07015C5DC1
:1046A0000A01E16F000E07015D590A01E26F000E79
:1046B00007015E590A01E36F000E07015F590A0105
:1046C000E46F07016051200DF3500A01E15F000E15
:1046D000E25BE35BE45BE4CAEAFAE3CAE9FAE2CA52
:1046E000E8FAE1CAE7FA00011AEC1EF003C0E4FAA6
:1046F00002C0E3FA01C0E2FA00C0E1FA0A01E153A4
:10470000D8A4DED1E253D8A4DBD1E353D8A4D8D1C6
:10471000E453D8A4D5D1060E07015C5D0A01E16F10
:10472000000E07015D590A01E26F000E07015E5994
:104730000A01E36F000E07015F590A01E46F0701E8
:104740006051200DF3500A01E15F000EE25BE35B74
:10475000E45BE4CAEAFAE3CAE9FAE2CAE8FAE1CABF
:10476000E7FA00011AEC1EF003C0E4FA02C0E3FA13
:1047700001C0E2FA00C0E1FA0A01E153D8A4A0D1D5
:10478000E253D8A49DD1E353D8A49AD1E453D8A43A
:1047900097D1150E07015C5D0A01E16F000E07015C
:1047A0005D590A01E26F000E07015E590A01E36FCD
:1047B000000E07015F590A01E46F07016051200DE7
:1047C000F3500A01E15F000EE25BE35BE45BE4CAE5
:1047D000EAFAE3CAE9FAE2CAE8FAE1CAE7FA00014A
:1047E0001AEC1EF003C0E4FA02C0E3FA01C0E2FAD8
:1047F00000C0E1FA0A0100500F08D8A461D1E253C9
:10480000D8A45ED1E353D8A45BD1E453D8A458D143
:10481000010E070160276051200DF3505C5D626F4F
:10482000000E5D59636F000E5E59646F000E5F5994
:10483000656F010E605D0D0DF3CF61F76051200DC6
:10484000F3505C5D0A01E16F000E07015D590A013A
:10485000E26F000E07015E590A01E36F000E0701C7
:104860005F590A01E46FEA6FE3CAE9FAE2CAE8FABB
:10487000E1CAE7FA00011AEC1EF000C0DFFA0701F6
:104880006051200DF3505C5D0A01E16F000E0701DD
:104890005D590A01E26F000E07015E590A01E36FDC
:1048A000000E07015F590A01E46F0D0EE127000EAB
:1048B000E223E323E423E4CAEAFAE3CAE9FAE2CA18
:1048C000E8FAE1CAE7FA00011AEC1EF000C0E0FACB
:1048D0000A01DE6BDE5105083CE0070161510A0167
:1048E000DE25036A750F016E070E032201C0E1FA8F
:1048F00003C0E2FAD890DE35070162250A01E36FB2
:10490000000E070163210A01E46F000E0701642114
:104910000A01E56F000E070165210A01E66F010E2D
:10492000E327000EE423E523E623E6CAEAFAE5CA14
:10493000E9FAE4CAE8FAE3CAE7FA00011AEC1EF061
:10494000E2CAEAFFE1CAE9FF00C0EFFF0A01DE2B7D
:10495000C1D7050EDE6FDE510B083CE00701615147
:104960000A01DE25036A750F016E070E032201C0DE
:10497000E1FA03C0E2FAD890DE35070162250A01A8
:10498000E36F000E070163210A01E46F000E0701C7
:1049900064210A01E56F000E070165210A01E66F37
:1049A000040EE327000EE423E523E623E6CAEAFA31
:1049B000E5CAE9FAE4CAE8FAE3CAE7FA00011AEC40
:1049C0001EF0E2CAEAFFE1CAE9FF00C0EFFF0A01F8
:1049D000DE2BC1D70B0EDE6FDE510D083CE0070168
:1049E00061510A01DE25036A750F016E070E03226D
:1049F00001C0E1FA03C0E2FAD890DE350701622572
:104A00000A01E36F000E070163210A01E46F000E43
:104A1000070164210A01E56F000E070165210A0103
:104A2000E66F060EE327000EE423E523E623E6CA3D
:104A3000EAFAE5CAE9FAE4CAE8FAE3CAE7FA0001E1
:104A40001AEC1EF0E2CAEAFFE1CAE9FF00C0EFFF7C
:104A50000A01DE2BC1D707016051200DF3505C5DC8
:104A60000A01E16F000E07015D590A01E26F000EB5
:104A700007015E590A01E36F000E07015F590A0141
:104A8000E46FEA6FE3CAE9FAE2CAE8FAE1CAE7FAD0
:104A900000011AEC1EF003C0E4FA02C0E3FA01C000
:104AA000E2FA00C0E1FA0A01E4530AE1E35308E143
:104AB000E25306E1E1513F0803E30601EED50A01A6
:104AC000D3D10601FD53D8B4CDD1050E07015C5DED
:104AD0000A01E16F000E07015D590A01E26F000E45
:104AE00007015E590A01E36F000E07015F590A01D1
:104AF000E46F07016051200DF3500A01E15F000EE1
:104B0000E25BE35BE45BE4CAEAFAE3CAE9FAE2CA1D
:104B1000E8FAE1CAE7FA00018CEC1EF00152D8A4D1
:104B2000A2D1060E07015C5D0A01E16F000E0701CC
:104B30005D590A01E26F000E07015E590A01E36F39
:104B4000000E07015F590A01E46F07016051200D53
:104B5000F3500A01E15F000EE25BE35BE45BE4CA51
:104B6000EAFAE3CAE9FAE2CAE8FAE1CAE7FA0001B6
:104B70008CEC1EF00152D8A476D1150E07015C5DB5
:104B80000A01E16F000E07015D590A01E26F000E94
:104B900007015E590A01E36F000E07015F590A0120
:104BA000E46F07016051200DF3500A01E15F000E30
:104BB000E25BE35BE45BE4CAEAFAE3CAE9FAE2CA6D
:104BC000E8FAE1CAE7FA00018CEC1EF001500F0888
:104BD000D8A449D1010E070160276051200DF35080
:104BE0005C5D626F000E5D59636F000E5E59646F0D
:104BF000000E5F59656F010E605D0D0DF3CF61F71B
:104C00006051200DF3505C5D0A01E16F000E070159
:104C10005D590A01E26F000E07015E590A01E36F58
:104C2000000E07015F590A01E46FEA6FE3CAE9FA6F
:104C3000E2CAE8FAE1CAE7FA00018CEC1EF001C012
:104C4000DFFA07016051200DF3505C5D0A01E16F4E
:104C5000000E07015D590A01E26F000E07015E595F
:104C60000A01E36F000E07015F590A01E46F0D0EA0
:104C7000E127000EE223E323E423E4CAEAFAE3CACD
:104C8000E9FAE2CAE8FAE1CAE7FA00018CEC1EF0A0
:104C900001C0E0FA0A01DE6BDE5105083CE00701C5
:104CA00061510A01DE25036A750F016E070E0322AA
:104CB00001C0E1FA03C0E2FAD890DE3507016225AF
:104CC0000A01E36F000E070163210A01E46F000E81
:104CD000070164210A01E56F000E070165210A0141
:104CE000E66F010EE327000EE423E523E623E6CA80
:104CF000EAFAE5CAE9FAE4CAE8FAE3CAE7FA00011F
:104D00008CEC1EF0E2CAEAFFE1CAE9FF01C0EFFF46
:104D10000A01DE2BC1D7050EDE6FDE510B083CE029
:104D2000070161510A01DE25036A750F016E070E46
:104D3000032201C0E1FA03C0E2FAD890DE35070190
:104D400062250A01E36F000E070163210A01E46F87
:104D5000000E070164210A01E56F000E07016521BD
:104D60000A01E66F040EE327000EE423E523E623A1
:104D7000E6CAEAFAE5CAE9FAE4CAE8FAE3CAE7FAEF
:104D800000018CEC1EF0E2CAEAFFE1CAE9FF01C0B3
:104D9000EFFF0A01DE2BC1D70B0EDE6FDE510D08CF
:104DA0003CE0070161510A01DE25036A750F016EBF
:104DB000070E032201C0E1FA03C0E2FAD890DE3503
:104DC000070162250A01E36F000E070163210A0152
:104DD000E46F000E070164210A01E56F000E070170
:104DE00065210A01E66F060EE327000EE423E523A2
:104DF000E623E6CAEAFAE5CAE9FAE4CAE8FAE3CA47
:104E0000E7FA00018CEC1EF0E2CAEAFFE1CAE9FF12
:104E100001C0EFFF0A01DE2BC1D707016051200D51
:104E2000F3505C5D0A01E16F000E07015D590A0154
:104E3000E26F000E07015E590A01E36F000E0701E1
:104E40005F590A01E46FEA6FE3CAE9FAE2CAE8FAD5
:104E5000E1CAE7FA00018CEC1EF001503F0803E3C1
:104E6000060133D600010A01070EE26F750EE16FED
:104E70000001C6EC1FF001C0AEF70701AE510808F3
:104E80000FE3070E0A01E26F750EE16F070EE46F84
:104E9000660EE36FE66B0D0EE56F0001E3EC1FF0AD
:104EA000020107AB1DD03C0EF66E100EF76E150E0C
:104EB0000A01E16F0001B1EC0CF0070EEA6E660E1C
:104EC000E96E2CEC20F0200E9EA8FED7AD6E0A0EE7
:104ED0009EA8FED7AD6E0D0E9EA8FED7AD6E020148
:104EE00007AB1DD0580EF66E100EF76E140E0A01A9
:104EF000E16F0001B1EC0CF0070EEA6E750EE96E81
:104F00002CEC20F0200E9EA8FED7AD6E0A0E9EA8B7
:104F1000FED7AD6E0D0E9EA8FED7AD6E020107AB9B
:104F200023D0720EF66E100EF76E190E0A01E16FA5
:104F30000001B1EC0CF0410EE96E5FC7E4FA5EC708
:104F4000E3FA5DC7E2FA5CC7E1FA3FEC20F0200E1D
:104F50009EA8FED7AD6E0A0E9EA8FED7AD6E0D0EB2
:104F60009EA8FED7AD6E020107AB1FD0920EF66E63
:104F7000100EF76E100E0A01E16F0001B1EC0CF09B
:104F800060C7E1FA1B0E0A01E26F0001B5EC20F0E8
:104F9000200E9EA8FED7AD6E0A0E9EA8FED7AD6E5F
:104FA0000D0E9EA8FED7AD6E020108ADB3D007016D
:104FB000603D01D0ADD0020108BF25D0070160518E
:104FC000200DF3505C5D0A01E16F000E07015D5991
:104FD0000A01E26F000E07015E590A01E36F000E3D
:104FE00007015F590A01E46FE86FE3CAE7FAE2CA12
:104FF000E6FAE1CAE5FAE50EE96FEA6B0001F4ECC6
:1050000020F083D0020108AF80D007016051200D4D
:10501000F3505C5D0A01E16F000E07015D590A0162
:10502000E26F000E07015E590A01E36F000E0701EF
:105030005F590A01E46FE86FE3CAE7FAE2CAE6FAE9
:10504000E1CAE5FAE96B010EEA6F0001F4EC20F029
:10505000010E0A01DE6FDE511F082DE007016051CD
:10506000200DF3505C5D0A01E16F000E07015D59F0
:105070000A01E26F000E07015E590A01E36F000E9C
:1050800007015F590A01E46FDE51E127000EE223B8
:10509000E323E423E4CAE8FAE3CAE7FAE2CAE6FA59
:1050A000E1CAE5FAE96B020EEA6F0001F4EC20F0C8
:1050B0000A01DE2BD0D707016051200DF3505C5D53
:1050C0000A01E16F000E07015D590A01E26F000E4F
:1050D00007015E590A01E36F000E07015F590A01DB
:1050E000E46F1F0EE127000EE223E323E423E4CA6A
:1050F000E8FAE3CAE7FAE2CAE6FAE1CAE5FAE96BD6
:10510000030EEA6F0001F4EC20F00701600750D7AE
:105110000201089D0001000CEF5210E0EACFDEFA18
:10512000E9CFDDFAEFCFEAFA2AEC11F0DECAEAFFA6
:10513000DDCAE9FFE92AD8B4EA2AEED7000C01500B
:10514000DECAE3FA640E0A01E46F00019FEC20F06E
:1051500000C0DEFA0150300E08E10A01DFA310D0D2
:10516000DFB70ED0DFB9200E04D00A01DF97DF9938
:10517000DF81012601C0EAFA00012AEC11F00A01E0
:10518000DECAE3FA0A0EE46F00019FEC20F000C0D3
:10519000DEFA0150300E08E10A01DFB70BD0DFA1C3
:1051A00009D0DFB9200E0001012601C0EAFA2AEC7D
:1051B00011F00A01300EDE27DECAEAFA00012AECFD
:1051C00011F0000CE9500A01E26F3B0EE96F9A0EF4
:1051D000E86FCA0EE76FE66B0A0EE46FD8820A0E1C
:1051E000EA6EDE0EE96EE1CAF0FAE0CAEFFADFCA53
:1051F000EEFADECAEDFAE9CAF4FAE8CAF3FAE7CA47
:10520000F2FAE6CAF1FA00015AEC16F00150005227
:1052100013E10A01E451010AD8A402D000010CD024
:10522000E2510CE00F0BE45D01E010E2E2BF0ED0B2
:10523000E2BD04D0200E03D00A01E26B300E00263E
:1052400000C0EAFA00012AEC11F00A01D892E9CA7A
:10525000F0FAE8CAEFFAE7CAEEFAE6CAEDFAF46B3A
:10526000F36BF26B0A0EF16F00015AEC16F003C0FB
:10527000E9FA02C0E8FA01C0E7FA00C0E6FA0A015A
:10528000E42FACD70001000C0A01E56BE36B0A0EBA
:10529000E46FE26BE16BE06BDF6BDD51DE1105E18A
:1052A000006A016A026A036A3DD1E551E52B036A8F
:1052B000DD25E96EDE510320EA6EEFCFE6FAE65116
:1052C0002D080DE1010EE36FE551E52B036ADD25A5
:1052D000E96EDE510320EA6EEFCFE6FA0DD0E6511B
:1052E0002B080AE1E551E52B036ADD25E96EDE5165
:1052F0000320EA6EEFCFE6FAE6512F08D8B0FAD0D5
:10530000E6513908D8A0F6D0E651300821E1036A09
:10531000E551DD25E96EDE510320EA6EEF50780895
:105320000AE0036AE551DD25E96EDE510320EA6EED
:10533000EF5058080DE1100EE46FE52BE551E52B19
:10534000036ADD25E96EDE510320EA6EEFCFE6FA4F
:10535000E4510A0844E1E6512F0840E2E6513908D9
:105360003DE3D890DF35E86FE035E96FE135EA6F6E
:10537000E235EB6FDF35006EE035016EE135026E30
:10538000E235036E0036013602360336003601364A
:1053900002360336F80E0016E8510026E9510122C4
:1053A000EA510222EB51032203C0E2FA02C0E1FA01
:1053B00001C0E0FA00C0DFFA300EE65DDF27000E24
:1053C000E023E123E223E551E52B036ADD25E96EC5
:1053D000DE510320EA6EEFCFE6FABDD78BD0E45161
:1053E0001008D8A487D0E651600806E2E6517A0892
:1053F00003E3E651DF0B01D0E651E66FE6512F08DB
:1054000003E2E651390807E2E6514008D8B072D00D
:10541000E65146086FE3E6512F082DE2E6513908C0
:105420002AE3DF35E86FE035E96FE135EA6FE23511
:10543000EB6FE837E937EA37EB37E837E937EA3730
:10544000EB37E837E937EA37EB37F00EE817300E7D
:10545000E65DE825006E000EE921016E000EEA21EE
:10546000026E000EEB21E26F02C0E1FA01C0E0FA29
:1054700000C0DFFA2AD0DF35E86FE035E96FE135AB
:10548000EA6FE235EB6FE837E937EA37EB37E837B1
:10549000E937EA37EB37E837E937EA37EB37F00E29
:1054A000E817410EE65D0A0FE825006E000EE921BF
:1054B000016E000EEA21026E000EEB21E26F02C0C7
:1054C000E1FA01C0E0FA00C0DFFAE551E52B036A1A
:1054D000DD25E96EDE510320EA6EEF50E66F6008CD
:1054E00006E2E6517A0803E3E651DF0B01D0E6510C
:1054F000E66F84D7E4510A080DE1E32D0BD0DF1FDE
:10550000E01FE11FE21FDF2BD8B4E02BD8B4E12B62
:10551000D8B4E22BDFCA00F0E0CA01F0E1CA02F021
:10552000E2CA03F000011BEF33F0020107A707D026
:105530005C0EF66E0B0EF76E00012FEC0CF0060100
:10554000FC6BFB6BFA6BF96B010E0201876F866FC8
:10555000856B846B0F0E836FFF0E826F0A01766B73
:1055600002011B6B1A6B196B186B096B0A6B0A0132
:10557000546B536B526B516B02010E6B07A708D033
:10558000640EF66E0B0EF76E00012FEC0CF00201AC
:1055900031A710D0B4C650FAB3C64FFAB2C64EFA0D
:1055A000B1C64DFAC0C658FABFC657FABEC656FABB
:1055B000BDC655FAD4C675FAD3C674FAD2C673FA04
:1055C000D1C672FA0A01606B5F6B5E6B5D6B0201A4
:1055D00007A737D06C0EF66E0B0EF76E0B0E0A0196
:1055E000E16F0001B1EC0CF050CAE1FA570E0A016C
:1055F000E26F0001C6EC0CF04FCAE1FA570E0A0147
:10560000E26F0001C6EC0CF04ECAE1FA570E0A0137
:10561000E26F0001C6EC0CF04DCAE1FA570E0A0128
:10562000E26F0001C6EC0CF0200E9EA8FED7AD6E16
:105630000A0E9EA8FED7AD6E0D0E9EA8FED7AD6ECB
:10564000020107A737D0800EF66E0B0EF76E0F0E15
:105650000A01E16F0001B1EC0CF058CAE1FA570EF3
:105660000A01E26F0001C6EC0CF057CAE1FA570ECE
:105670000A01E26F0001C6EC0CF056CAE1FA570EBF
:105680000A01E26F0001C6EC0CF055CAE1FA570EB0
:105690000A01E26F0001C6EC0CF0200E9EA8FED7B6
:1056A000AD6E0A0E9EA8FED7AD6E0D0E9EA8FED75B
:1056B000AD6E020107A737D0980EF66E0B0EF76E8F
:1056C0000C0E0A01E16F0001B1EC0CF075CAE1FAB1
:1056D000570E0A01E26F0001C6EC0CF074CAE1FA41
:1056E000570E0A01E26F0001C6EC0CF073CAE1FA32
:1056F000570E0A01E26F0001C6EC0CF072CAE1FA23
:10570000570E0A01E26F0001C6EC0CF0200E9EA8B5
:10571000FED7AD6E0A0E9EA8FED7AD6E0D0E9EA8EA
:10572000FED7AD6E020131A716D0060191510A01D4
:1057300072257C6F060192510A0173217D6F06016B
:1057400093510A0174217E6F060194510A0175215B
:105750007F6F46D0020131B744D00601A5350A015A
:10576000DD6F0601A6350A01DE6F0601A7350A01C5
:10577000DF6F0601A8350A01E06FDD37DE37DF375E
:10578000E037DD37DE37DF37E037DD37DE37DF376D
:10579000E037DD37DE37DF37E037E00EDD17D89250
:1057A000E0CAF0FADFCAEFFADECAEEFADDCAEDFAB5
:1057B000B8C6F4FAB7C6F3FAB6C6F2FAB5C6F1FA45
:1057C00000015AEC16F000500A0172257C6F01505E
:1057D00073217D6F025074217E6F035075217F6F9E
:1057E000020107A72FD0AC0EF66E0B0EF76E0C0E53
:1057F0000A01E16F0001B1EC0CF075CAE1FA570E35
:105800000A01E26F0001C6EC0CF074CAE1FA570E0F
:105810000A01E26F0001C6EC0CF073CAE1FA570E00
:105820000A01E26F0001C6EC0CF072CAE1FA570EF1
:105830000A01E26F0001C6EC0CF0200E9EA8FED714
:10584000AD6E020107A734D0BE0EF66E0B0EF76EDA
:105850000A0E0A01E16F0001B1EC0CF07FCAE1FA17
:10586000570E0A01E26F0001C6EC0CF07ECAE1FAA5
:10587000570E0A01E26F0001C6EC0CF07DCAE1FA96
:10588000570E0A01E26F0001C6EC0CF07CCAE1FA87
:10589000570E0A01E26F0001C6EC0CF0CC0EF66E5A
:1058A0000B0EF76E040E0A01E16F0001B1EC0CF073
:1058B00075CA4CFA74CA4BFA73CA4AFA72CA49FAE0
:1058C0000A017C51495D0BE17D514A5D08E17E5141
:1058D0004B5D05E17F514C5DD8B4AAEF36F0020173
:1058E00007A7CDD0D20EF66E0B0EF76E0A0E0A0188
:1058F000E16F0001B1EC0CF04CCAE1FA570E0A015D
:10590000E26F0001C6EC0CF04BCAE1FA570E0A0137
:10591000E26F0001C6EC0CF04ACAE1FA570E0A0128
:10592000E26F0001C6EC0CF049CAE1FA570E0A0119
:10593000E26F0001C6EC0CF0200E9EA8FED7AD6E03
:10594000E20EF66E0B0EF76E080E0A01E16F000113
:10595000B1EC0CF05CCAE1FA570E0A01E26F0001EB
:10596000C6EC0CF05BCAE1FA570E0A01E26F0001C7
:10597000C6EC0CF05ACAE1FA570E0A01E26F0001B8
:10598000C6EC0CF059CAE1FA570E0A01E26F0001A9
:10599000C6EC0CF0200E9EA8FED7AD6EF00EF66E93
:1059A0000B0EF76E090E0A01E16F0001B1EC0CF06D
:1059B00060CAE1FA570E0A01E26F0001C6EC0CF072
:1059C0005FCAE1FA570E0A01E26F0001C6EC0CF063
:1059D0005ECAE1FA570E0A01E26F0001C6EC0CF054
:1059E0005DCAE1FA570E0A01E26F0001C6EC0CF045
:1059F000200E9EA8FED7AD6E0A017651040DF3501D
:105A0000036A8D0FE96E0A0E0320EA6EEFCFDDFA0E
:105A1000ECCFDEFAECCFDFFAECCFE0FAFE0EF66E5A
:105A20000B0EF76E090EE16F0001B1EC0CF0E0CA4D
:105A3000E1FA570E0A01E26F0001C6EC0CF0DFCA72
:105A4000E1FA570E0A01E26F0001C6EC0CF0DECA63
:105A5000E1FA570E0A01E26F0001C6EC0CF0DDCA54
:105A6000E1FA570E0A01E26F0001C6EC0CF00A0ED3
:105A70009EA8FED7AD6E0D0E9EA8FED7AD6E0A0194
:105A800059530BE15A51020808E15B5306E15C539C
:105A900004E1606B5F6B5E6B5D6B4CCA0BFD4BCAC8
:105AA0000AFD4ACA09FD49CA08FD080E0D010D6F1D
:105AB000490E0C6F000197EC15F060CA5CFA5FCAE2
:105AC0005BFA5ECA5AFA5DCA59FA0A01595309E1EA
:105AD0005A51020806E15B5304E15C53D8B4A0EFCD
:105AE00036F0490E5925E96E080E5A21EA6EEF503C
:105AF0007F0810E2020107A708D00E0EF66E0C0E0A
:105B0000F76E00012FEC0CF0020197EF36F090EFEA
:105B100031F00A010B0E5925DD6F000E5A21DE6FA0
:105B2000000E5B21DF6F000E5C21E06F490EDD256A
:105B3000E96E080EDE21EA6EEF500C0B0C0810E146
:105B4000020107A708D0140EF66E0C0EF76E0001C6
:105B50002FEC0CF0020197EF36F090EF31F00A01D4
:105B6000490E5925E96E080E5A21EA6EEF52D8A463
:105B700080D0020107A707D01A0EF66E0C0EF76E42
:105B800000012FEC0CF00A017651000861E20201DD
:105B900007A707D0200EF66E0C0EF76E00012FEC53
:105BA0000CF00A017607010E02010A270A0176515C
:105BB000040DF350036A8D0FE96E0A0E0320EA6E9E
:105BC000EFCF00F0ECCF01F0ECCF02F0ECCF03F020
:105BD00003C060FA02C05FFA01C05EFA00C05DFA5D
:105BE0007651040DF350036AB50FE96E0A0E0320D7
:105BF000EA6EEFCF00F0ECCF01F0ECCF02F0ECCF8B
:105C000003F003C075FA02C074FA01C073FA00C051
:105C100072FA200E5D27000E5E235F2360235D5322
:105C200013E15E51020810E15F530EE160530CE195
:105C3000010E7227D8B0732BD8B4742BD8B4752B3F
:105C4000606B5F6B5E6B5D6B02016DD510D00A01FE
:105C500076530EE1020107A508D0260EF66E0C0E53
:105C6000F76E00012FEC0CF0020157EF3AF00A0139
:105C700058D30B0E5925DD6F000E5A21DE6F000E32
:105C80005B21DF6F000E5C21E06F490EDD25E96EC0
:105C9000080EDE21EA6EEF501C0B1008D8A441D389
:105CA000020107A507D02C0EF66E0C0EF76E000150
:105CB0002FEC0CF0490E0A015925E96E080E5A2105
:105CC000EA6EEF502E0803E1020197EF36F008016B
:105CD000445304E102010F2B1CD008014451020877
:105CE00018E102010E2B0E510D5D13E1010E182576
:105CF0001C6F000E19211D6F000E1A211E6F000E61
:105D00001B211F6F0891010E0801446F020157EF1C
:105D10003AF00A017651040DF350036A8D0FE96ED3
:105D20000A0E0320EA6E59CAEFFF5ACAECFF5BCA9B
:105D3000ECFF5CCAECFF7651040DF350036AB50F1B
:105D4000E96E0A0E0320EA6E49CAEFFF4ACAECFF69
:105D50004BCAECFF4CCAECFF762B0201092B036AFD
:105D60000951230FE96E070E0320EA6E76CAEFFF92
:105D70000A6B080144510308D8A42ED102010D5327
:105D800002E1010E0D6F0E2B0D510E5DD8A099D0C2
:105D90000A017651000867E24CCAE4FA4BCAE3FAFA
:105DA0004ACAE2FA49CAE1FAB8C6E8FAB7C6E7FA57
:105DB000B6C6E6FAB5C6E5FA00012CEC16F00A0103
:105DC0005951002407015C6F0A015A510120070153
:105DD0005D6F0A015B51022007015E6F0A015C5191
:105DE000032007015F6F000127EC22F0020107A7E3
:105DF0001DD0320EF66E0C0EF76E040E0A01E16F26
:105E00000001B1EC0CF0070EEA6E750EE96E2CEC99
:105E100020F0200E9EA8FED7AD6E0A0E9EA8FED7DB
:105E2000AD6E0D0E9EA8FED7AD6E0201070EEA6E96
:105E30009D0EE96E000E000181EC03F00A000900DE
:105E4000F550EE6E0009FBE1070E0A01E26F9D0EB0
:105E5000E16F070EE46F750EE36FE66B100EE56FF2
:105E60000001E3EC1FF002012851080DF3CFDDFA29
:105E70000A01DE6BDDCADFFA0001C2EC0EF002019E
:105E8000285306E10F0E856F846B836FFF0E826FC0
:105E900007A708D03C0EF66E0C0EF76E00012FEC33
:105EA0000CF00201070EEA6E9D0EE96E00018CEC0B
:105EB00028F00201856B846B0F0E836FFF0E826FDB
:105EC000282B060E0D250E5D04E00F510E5DD8A4A3
:105ED00082D00A01DE6B380EDF6F0001C2EC0EF0DB
:105EE000020108AB0FD00F0E856F846F836B826B3E
:105EF000440EF66E0C0EF76E00016AEC11F0020112
:105F000057EF3AF0856B846B836BFF0E826F560EF2
:105F1000F66E0C0EF76E00016AEC11F00DC2DEFA9F
:105F2000010E0A01DF6F00019FEC28F02F0E0A011D
:105F3000EA6F00012AEC11F00FC2DEFA010E0A012D
:105F4000DF6F00019FEC28F0200E0A01EA6F0001CC
:105F50002AEC11F0200E0A01EA6F00012AEC11F080
:105F6000200E0A01EA6F00012AEC11F00201856B94
:105F7000846B0F0E836FF00E826F580EF66E0C0E50
:105F8000F76E00016AEC11F0036A02010D51FE0F79
:105F9000E96E060E0320EA6EEFCFDDFADDCADEFA07
:105FA000010E0A01DF6F00019FEC28F02F0E0A019D
:105FB000EA6F00012AEC11F0430EE96E17C2E1FA14
:105FC00016C2E0FA15C2DFFA14C2DEFAE2EC28F0DB
:105FD000020157EF3AF00801442D00D0020107A753
:105FE00008D05A0EF66E0C0EF76E00012FEC0CF076
:105FF000020107A759D0600EF66E0C0EF76E040E64
:106000000A01E16F0001B1EC0CF009C2E1FA1B0ECC
:106010000A01E26F0001B5EC20F0200E9EA8FED729
:10602000AD6E200E9EA8FED7AD6E6A0EF66E0C0EFB
:10603000F76E0A0E0A01E16F0001B1EC0CF076CAAE
:10604000E1FA1B0E0A01E26F0001B5EC20F0200E10
:106050009EA8FED7AD6E200E9EA8FED7AD6E0A019B
:10606000765100080AE276CA77FA775306E02E0ED8
:106070009EA8FED7AD6E7707F8D75C0E9EA8FED718
:10608000AD6E0A0EEA6E800EE96E00012CEC20F077
:10609000200E9EA8FED7AD6E0A0E9EA8FED7AD6E4E
:1060A0000D0E9EA8FED7AD6E150E0A015925DD6FA7
:1060B000000E5A21DE6F000E5B21000E5C21490E9E
:1060C000DD25E96E080EDE21EA6EEFCF45F8080106
:1060D0000A017B6B7A6B796B45C878FA7ACA7BFACE
:1060E00079CA7AFA78CA79FA786B140E5925DD6F75
:1060F000000E5A21DE6F000E5B21000E5C21490E5E
:10610000DD25E96E080EDE21EA6EEFCF46F80801C4
:1061100046510A017827000E79237A237B237ACA15
:106120007BFA79CA7AFA78CA79FA786B1B0E592504
:10613000DD6F000E5A21DE6F000E5B21000E5C2128
:10614000490EDD25E96E080EDE21EA6EEFCF47F835
:10615000080147510A017827000E79237A237B230F
:106160007ACA7BFA79CA7AFA78CA79FA786B1A0EFF
:106170005925DD6F000E5A21DE6F000E5B21000EE7
:106180005C21490EDD25E96E080EDE21EA6EEFCFB7
:1061900048F8080148510A017827000E79237A232C
:1061A0007B23020107AB36D07A0EF66E0C0EF76E2B
:1061B000090E0A01E16F0001B1EC0CF07BCAE1FAB3
:1061C000570E0A01E26F0001C6EC0CF07ACAE1FA40
:1061D000570E0A01E26F0001C6EC0CF079CAE1FA31
:1061E000570E0A01E26F0001C6EC0CF078CAE1FA22
:1061F000570E0A01E26F0001C6EC0CF0200E9EA8BB
:10620000FED7AD6E0A0E9EA8FED7AD6E0D0E9EA8EF
:10621000FED7AD6E020E0A01785F000E795B7A5BE5
:106220007B5B020107AB36D08C0EF66E0C0EF76E60
:10623000090E0A01E16F0001B1EC0CF07BCAE1FA32
:10624000570E0A01E26F0001C6EC0CF07ACAE1FABF
:10625000570E0A01E26F0001C6EC0CF079CAE1FAB0
:10626000570E0A01E26F0001C6EC0CF078CAE1FAA1
:10627000570E0A01E26F0001C6EC0CF0200E9EA83A
:10628000FED7AD6E0A0E9EA8FED7AD6E0D0E9EA86F
:10629000FED7AD6E7BCAE4FA7ACAE3FA79CAE2FAAB
:1062A00078CAE1FA94C6E8FA93C6E7FA92C6E6FA23
:1062B00091C6E5FA00012CEC16F003C075FA02C095
:1062C00074FA01C073FA00C072FA0601D5510A01CE
:1062D00072270601D6510A0173230601D7510A011C
:1062E00074230601D8510A017523020131A710D089
:1062F000060191510A01725F060192510A01735B16
:10630000060193510A01745B060194510A01755B01
:106310000A01606B5F6B5E6B5D6B020193EF2BF0AC
:106320000A01080E5925DD6F000E5A21DE6F000E9E
:106330005B21000E5C21490EDD25E96E080EDE2191
:10634000EA6EEFCF61FA090E5925DD6F000E5A2172
:10635000DE6F000E5B21000E5C21490EDD25E96E2B
:10636000080EDE21EA6EEFCF62FA0A0E5925DD6FC4
:10637000000E5A21DE6F000E5B21000E5C21490EDB
:10638000DD25E96E080EDE21EA6EEFCF63FA61517A
:106390006D0811E061514D080EE0615177080BE086
:1063A0006151570808E061516F0805E061514F08DD
:1063B000D8A496EF36F0625170081DE06251500883
:1063C0001AE06251610817E06251410814E062511D
:1063D000670811E0625147080EE062516D080BE05A
:1063E00062514D0808E06251690805E062514908B0
:1063F000D8A496EF36F0635133081AE0635176085B
:1064000017E06351560814E06351670811E06351C7
:1064100047080EE0635161080BE06351410808E052
:106420006351640805E063514408D8A496EF36F040
:1064300008014453D8A42BD1010E02011427D8B06F
:10644000152BD8B4162BD8B4172B07A714D09E0E33
:10645000F66E0C0EF76E00012FEC0CF014C2E1FA90
:10646000570E0A01E26F0001C6EC0CF0200E9EA848
:10647000FED7AD6E020107A716D0A80EF66E0C0E61
:10648000F76E0B0E0A01E16F0001B1EC0CF009C2CE
:10649000E1FA570E0A01E26F0001C6EC0CF0200E83
:1064A0009EA8FED7AD6E0A01765321E002010A5381
:1064B0000FE00A51095D036A230FE96E070E0320FE
:1064C000EA6EEF500A01765D04E202010A2BF1D771
:1064D0000A0102010A51095D036AFE0FE96E060E08
:1064E0000320EA6E010EEF24EF6E06D00A01765308
:1064F00003E1010E0601FE27490E0A015925E96E46
:10650000080E5A21EA6EEFCF64FA010E5925DD6FAD
:10651000000E5A21DE6F000E5B21000E5C21490E39
:10652000DD25E96E080EDE21EA6EEFCF65FA020E78
:106530005925DD6F000E5A21DE6F000E5B21000E23
:106540005C21490EDD25E96E080EDE21EA6EEFCFF3
:1065500066FA030E5925DD6F000E5A21DE6F000E1C
:106560005B21000E5C21490EDD25E96E080EDE215F
:10657000EA6EEFCF67FA64515208D8A486D065510D
:106580004508D8A482D066514308D8A47ED067516C
:106590002D08D8A47AD0040E5925DD6F000E5A219B
:1065A000DE6F000E5B21000E5C21490EDD25E96ED9
:1065B000080EDE21EA6EEFCF68FA050E5925DD6F71
:1065C000000E5A21DE6F000E5B21000E5C21490E89
:1065D000DD25E96E080EDE21EA6EEFCF69FA060EC0
:1065E0005925DD6F000E5A21DE6F000E5B21000E73
:1065F0005C21490EDD25E96E080EDE21EA6EEFCF43
:106600006AFA070E5925DD6F000E5A21DE6F000E63
:106610005B21000E5C21490EDD25E96E080EDE21AE
:10662000EA6EEFCF6BFA6C6B0A0EDE6F680EDD6FF1
:10663000000144EF29F003C071FA02C070FA01C0F2
:106640006FFA00C06EFA0601FC510A01715D1DE38C
:1066500014E10601FB510A01705D17E30EE106012A
:10666000FA510A016F5D11E308E16E510601F95D0F
:10667000D8A002D00A0109D00A0171CAFCF670CA7A
:10668000FBF66FCAFAF66ECAF9F650D30801442D2C
:1066900040D3010E02011827D8B0192BD8B41A2BF9
:1066A000D8B41B2B08A5A5D11F511B5DD8A0A1D123
:1066B0000EE11E511A5DD8A09CD109E11D51195D52
:1066C000D8A097D104E11C51185DD8A092D1036ADB
:1066D0000D51FE0FE96E060E0320EA6EEF5232E115
:1066E0000A01DE6B180EDF6F0001C2EC0EF0010E26
:1066F0000201876F866F856B846B0F0E836FF00EC0
:10670000826FB80EF66E0C0EF76E00016AEC11F097
:10671000020108AB15D00A01DE6B380EDF6F0001F5
:10672000C2EC0EF00F0E0201856F846F836B826BDB
:10673000C80EF66E0C0EF76E00016AEC11F0020145
:1067400057EF3AF04CCAE4FA4BCAE3FA4ACAE2FA03
:1067500049CAE1FAB8C6E8FAB7C6E7FAB6C6E6FA31
:10676000B5C6E5FA00012CEC16F00A0159510024D7
:1067700007015C6F0A015A51012007015D6F0A0190
:106780005B51022007015E6F0A015C510320070183
:106790005F6F000127EC22F0070EEA6E9D0EE96E96
:1067A000000E8AEC03F00A000900F550EE6E0009B5
:1067B000FBE10701AD6B070E0A01E26F9D0EE16F71
:1067C000070EE46F750EE36FE66B100EE56F0001C8
:1067D000E3EC1FF002012951080DF3CFDDFA0A01A5
:1067E000DE6BDDCADFFA0001C2EC0EF002012953B4
:1067F00006E10F0E856F846B836FFF0E826F070EAD
:10680000EA6E9D0EE96E00018CEC28F00201856BAA
:10681000846B0F0E836FFF0E826F292B060E1C25D3
:10682000006E000E1D21016E000E1E21026E000E74
:106830001F21036E0050185D09E10150195D06E14A
:1068400002501A5D03E103501B5D57E0036A0D51CE
:10685000FE0FE96E060E0320EA6EEF502025006E53
:10686000000E2121016E000E2221026E000E232156
:10687000036E1F5D0CE341E102501E5D08E33DE144
:1068800001501D5D04E339E100501C5D36E2036AEE
:106890000D51FE0FE96E060E0320EA6EEF50202523
:1068A0000A01DD6F000E020121210A01DE6F000ED8
:1068B000020122210A01DF6F000E020123210A01D9
:1068C000E06F010EDD5D006E000EDE59016E000E00
:1068D000DF59026E000EE059036E00500201185D90
:1068E000D8A487D00150195DD8A483D002501A5D76
:1068F000D8A47FD003501B5D7CE10A01DE6B380E0B
:10690000DF6F0001C2EC0EF0020108AB0FD00F0EDA
:10691000856F846F836B826BDA0EF66E0C0EF76EEA
:1069200000016AEC11F0020157EF3AF0856B846BBD
:106930000F0E836FF00E826FEC0EF66E0C0EF76E7C
:1069400000016AEC11F0430EE96E1FC2E1FA1EC2AB
:10695000E0FA1DC2DFFA1CC2DEFAE2EC28F02F0ECC
:106960000A01EA6F00012AEC11F0430EE96E17C22A
:10697000E1FA16C2E0FA15C2DFFA14C2DEFAE2EC5E
:1069800028F0200E0A01EA6F00012AEC11F0200E17
:106990000A01EA6F00012AEC11F00201856B846B99
:1069A000836BFF0E826FEE0EF66E0C0EF76E00011B
:1069B0006AEC11F00DC2DEFA010E0A01DF6F000170
:1069C0009FEC28F02F0E0A01EA6F00012AEC11F06B
:1069D0000FC2DEFA010E0A01DF6F00019FEC28F002
:1069E0000201856B846B0F0E836FFF0E826F57EF72
:1069F0003AF018511C5DD8A48AD119511D5DD8A454
:106A000086D11A511E5DD8A482D11B511F5DD8A416
:106A10007ED108B57CD1150E0A015925DD6F000E17
:106A20005A21DE6F000E5B21000E5C21490EDD2530
:106A3000E96E080EDE21EA6EEFCF45F80801060187
:106A4000E06BDF6BDE6B45C8DDF6DFC6E0F6DEC669
:106A5000DFF6DDC6DEF6DD6B140E0A015925DD6FAB
:106A6000000E5A21DE6F000E5B21000E5C21490EE4
:106A7000DD25E96E080EDE21EA6EEFCF46F808014B
:106A800046510601DD27000EDE23DF23E023DFC6AB
:106A9000E0F6DEC6DFF6DDC6DEF6DD6B1B0E0A01B4
:106AA0005925DD6F000E5A21DE6F000E5B21000EAE
:106AB0005C21490EDD25E96E080EDE21EA6EEFCF7E
:106AC00047F8080147510601DD27000EDE23DF23CA
:106AD000E023DFC6E0F6DEC6DFF6DDC6DEF6DD6B00
:106AE0001A0E0A015925DD6F000E5A21DE6F000EC5
:106AF0005B21000E5C21490EDD25E96E080EDE21CA
:106B0000EA6EEFCF48F8080148510601DD27000E74
:106B1000DE23DF23E023020EDD5D0A01DD6F000EC0
:106B20000601DE590A01DE6F000E0601DF590A0177
:106B3000DF6F000E0601E0590A01E06FE46FDFCA63
:106B4000E3FADECAE2FADDCAE1FA94C6E8FA93C6CD
:106B5000E7FA92C6E6FA91C6E5FA00012CEC16F0C7
:106B600003C04BF702C04AF701C049F700C048F71D
:106B70000601D551070148270601D65107014923CF
:106B80000601D75107014A230601D85107014B23BB
:106B9000020131A710D0060191510701485F06019B
:106BA00092510701495B0601935107014A5B0601B7
:106BB000945107014B5B1F0E0A015925DD6F000E32
:106BC0005A21DE6F000E5B21000E5C21490EDD258F
:106BD000E96E080EDE21EA6EEFCF45F808010601E6
:106BE000EC6BEB6BEA6B45C8E9F6EBC6ECF6EAC674
:106BF000EBF6E9C6EAF6E96B1E0E0A015925DD6FD0
:106C0000000E5A21DE6F000E5B21000E5C21490E42
:106C1000DD25E96E080EDE21EA6EEFCF46F80801A9
:106C200046510601E927000EEA23EB23EC23EBC6CD
:106C3000ECF6EAC6EBF6E9C6EAF6E96B1D0E0A01C8
:106C40005925DD6F000E5A21DE6F000E5B21000E0C
:106C50005C21490EDD25E96E080EDE21EA6EEFCFDC
:106C600047F8080147510601E927000EEA23EB2304
:106C7000EC23EBC6ECF6EAC6EBF6E9C6EAF6E96BFE
:106C80001C0E0A015925DD6F000E5A21DE6F000E21
:106C90005B21000E5C21490EDD25E96E080EDE2128
:106CA000EA6EEFCF48F8080148510601E927000EC7
:106CB000EA23EB23EC234CCAE4FA4BCAE3FA4ACAB0
:106CC000E2FA49CAE1FAB8C6E8FAB7C6E7FAB6C6C0
:106CD000E6FAB5C6E5FA00012CEC16F00A015951A6
:106CE000002407015C6F0A015A51012007015D6F02
:106CF0000A015B51022007015E6F0A015C5103200B
:106D000007015F6F000127EC22F00201D0D30DD004
:106D100008014451020809E1010E02011827D8B008
:106D2000192BD8B41A2BD8B41B2B0A010201200E40
:106D30000A015927000E5A235B235C2366EF2DF0CE
:106D4000010E4927D8B04A2BD8B44B2BD8B44C2BC2
:106D500061EF2CF00601CD510A01725DDD6F060175
:106D6000CE510A017359DE6F0601CF510A017459E1
:106D7000DF6F0601D0510A017559E06FD890060106
:106D80009135006E9235016E9335026E9435036E27
:106D900000500A01DD270150DE230250DF2303509B
:106DA000E023D892E0CAF0FADFCAEFFADECAEEFAC0
:106DB000DDCAEDFA94C6F4FA93C6F3FA92C6F2FA73
:106DC00091C6F1FA00015AEC16F003C058FA02C05D
:106DD00057FA01C056FA00C055FA020131B73CD04B
:106DE000D8900601B831036EB731026EB631016E2C
:106DF000B531006E03C0E0FA02C0DFFA01C0DEFA6E
:106E0000E8CFDDFAD89258CAF0FA57CAEFFA56CA54
:106E1000EEFA55CAEDFA03C0F4FA02C0F3FA01C063
:106E2000F2FAE8CFF1FA00015AEC16F00601B1517E
:106E30000A0100244D6F0601B2510A0101204E6F74
:106E40000601B3510A0102204F6F0601B4510A0135
:106E50000320506F42D0020131A740D00601B83163
:106E6000036EB731026EB631016EB531006E03327A
:106E70000232013200323F0E031603C0E0FA02C0B4
:106E8000DFFA01C0DEFA00C0DDFAD89258CAF0FA83
:106E900057CAEFFA56CAEEFA55CAEDFA03C0F4FA29
:106EA00002C0F3FA01C0F2FA00C0F1FA00015AEC94
:106EB00016F00601B1510A0100244D6F0601B251CE
:106EC0000A0101204E6F0601B3510A0102204F6FE3
:106ED0000601B4510A010320506F020131B72ED1CF
:106EE000F00EF66E0C0EF76E00012FEC0CF050CA8F
:106EF0000BFD4FCA0AFD4ECA09FD4DCA08FD080E1A
:106F00000D010D6F490E0C6F000197EC15F00A0191
:106F1000E06B006A0050555DDD6F56515659DE6FCB
:106F200057515759DF6F58515859E06FD890DD3598
:106F3000596FDE355A6FDF355B6FE0355C6F010EE0
:106F40005925DD6F000E5A21DE6F000E5B21000E09
:106F50005C21490EDD25E96E080EDE21EA6EEFCFD9
:106F600045F808010A01546B536B526B45C851FA3E
:106F700053CA54FA52CA53FA51CA52FA516B490EC3
:106F80005925E96E080E5A21EA6EEFCF46F808013E
:106F900046510A015127000E5223532354235453C0
:106FA0000CE153530AE15251FE08D8B0C6D0FF0A93
:106FB00004E15151EF08D8B0C0D0020107A737D083
:106FC000FA0EF66E0C0EF76E0C0E0A01E16F000160
:106FD000B1EC0CF054CAE1FA570E0A01E26F00015D
:106FE000C6EC0CF053CAE1FA570E0A01E26F000139
:106FF000C6EC0CF052CAE1FA570E0A01E26F00012A
:10700000C6EC0CF051CAE1FA570E0A01E26F00011A
:10701000C6EC0CF0200E9EA8FED7AD6E0A0E9EA800
:10702000FED7AD6E0D0E9EA8FED7AD6E0201D890B4
:107030000601B831036EB731026EB631016EB5315B
:10704000006E03C0E0FA02C0DFFA01C0DEFAE8CF4A
:10705000DDFAD89254CAF0FA53CAEFFA52CAEEFADD
:1070600051CAEDFA03C0F4FA02C0F3FA01C0F2FA11
:10707000E8CFF1FA00015AEC16F00601B1510A010D
:1070800000244D6F0601B2510A0101204E6F060126
:10709000B3510A0102204F6F0601B4510A010320C7
:1070A000506F54CA58FA53CA57FA52CA56FA51CABC
:1070B00055FA58CAE4FA57CAE3FA56CAE2FA55CA68
:1070C000E1FA94C6E8FA93C6E7FA92C6E6FA91C6E0
:1070D000E5FA00012CEC16F003C0E0FA02C0DFFA7A
:1070E00001C0DEFA00C0DDFA0601CD510A01DD273C
:1070F0000601CE510A01DE230601CF510A01DF232A
:107100000601D0510A01E023D89006019135006EA6
:107110009235016E9335026E9435036E00500A016C
:10712000DD5D726F0150DE59736F0250DF59746F6D
:107130000350E059756FE7EF2AF0020131A7B7D18C
:107140000E0EF66E0D0EF76E00012FEC0CF050CA0D
:107150000BFD4FCA0AFD4ECA09FD4DCA08FD080EB7
:107160000D010D6F490E0C6F000197EC15F00A012F
:107170005831E06F5731DF6F5631DE6F5531DD6FBB
:10718000E033DF33DE33DD33E033DF33DE33DD3373
:10719000E033DF33DE33DD33E033DF33DE33DD3363
:1071A000E033DF33DE33DD33E033DF33DE33DD3353
:1071B000010EE017DD35006EDE35016EDF35026E43
:1071C000E035036E003601360236033600360136EE
:1071D00002360336003601360236033600360136F3
:1071E00002360336003601360236033600360136E3
:1071F00002360336800E00160050555DDD6F0150DB
:107200005659DE6F02505759DF6F03505859E06FDF
:10721000DD35596FDE355A6FDF355B6FE0355C6FFA
:1072200059375A375B375C37FC0E5917030E59250F
:10723000DD6F000E5A21DE6F000E5B21000E5C2117
:10724000490EDD25E96E080EDE21EA6EEFCF45F826
:1072500008010A01546B536B526B45C851FA53CA6B
:1072600054FA52CA53FA51CA52FA516B020E5925B6
:10727000DD6F000E5A21DE6F000E5B21000E5C21D7
:10728000490EDD25E96E080EDE21EA6EEFCF46F8E5
:10729000080146510A015127000E5223532354235B
:1072A00053CA54FA52CA53FA51CA52FA516B010ED8
:1072B0005925DD6F000E5A21DE6F000E5B21000E96
:1072C0005C21490EDD25E96E080EDE21EA6EEFCF66
:1072D00047F8080147510A015127000E5223532352
:1072E000542353CA54FA52CA53FA51CA52FA516B30
:1072F000490E5925E96E080E5A21EA6EEFCF48F87B
:10730000080148510A015127000E522353235423E8
:10731000513D08D0523D06D0533D04D054510F0882
:10732000D8B4C4D0020107A736D0180EF66E0D0EE1
:10733000F76E0C0E0A01E16F0001B1EC0CF054CABB
:10734000E1FA570E0A01E26F0001C6EC0CF053CAD5
:10735000E1FA570E0A01E26F0001C6EC0CF052CAC6
:10736000E1FA570E0A01E26F0001C6EC0CF051CAB7
:10737000E1FA570E0A01E26F0001C6EC0CF0200E94
:107380009EA8FED7AD6E0A0E9EA8FED7AD6E0D0E5E
:107390009EA8FED7AD6E0601B831036EB731026EFE
:1073A000B631016EB531006E033202320132003265
:1073B0003F0E031603C0E0FA02C0DFFA01C0DEFA96
:1073C00000C0DDFAD89254CAF0FA53CAEFFA52CA92
:1073D000EEFA51CAEDFA03C0F4FA02C0F3FA01C0A2
:1073E000F2FA00C0F1FA00015AEC16F00601B151B0
:1073F0000A0100244D6F0601B2510A0101204E6FAF
:107400000601B3510A0102204F6F0601B4510A016F
:107410000320506F54CA58FA53CA57FA52CA56FA40
:1074200051CA55FA58CAE4FA57CAE3FA56CAE2FAF8
:1074300055CAE1FA94C6E8FA93C6E7FA92C6E6FAA4
:1074400091C6E5FA00012CEC16F003C0E0FA02C088
:10745000DFFA01C0DEFA00C0DDFA0601CD510A01F3
:10746000DD270601CE510A01DE230601CF510A01B4
:10747000DF230601D0510A01E023D890060191359F
:10748000006E9235016E9335026E9435036E005096
:107490000A01DD5D726F0150DE59736F0250DF59D2
:1074A000746F0350E059756FE7EF2AF00201000195
:1074B000000CA3EF12F0020107A507D0EC0EF66E48
:1074C000160EF76E00012FEC0CF00001A4EF16F081
:1074D000020107A508D0000EF66E170EF76E000128
:1074E0002FEC0CF00201079D176B166B156B146BDC
:1074F0001F6B1E6B1D6B010E1C6F0B6B0D6B0F6BEF
:107500000801436B4351230812E0036A4351FE0F05
:10751000E96E060E0320EA6EEF6A036A4351230FF9
:10752000E96E070E0320EA6EEF6A432BEBD7446B3C
:10753000000195EC2AF0020107A537D01A0EF66E6D
:10754000170EF76E0D0E0A01E16F0001B1EC0CF0A1
:1075500017C2E1FA570E0A01E26F0001C6EC0CF007
:1075600016C2E1FA570E0A01E26F0001C6EC0CF0F8
:1075700015C2E1FA570E0A01E26F0001C6EC0CF0E9
:1075800014C2E1FA570E0A01E26F0001C6EC0CF0DA
:10759000200E9EA8FED7AD6E0A0E9EA8FED7AD6E39
:1075A0000D0E9EA8FED7AD6E020107A547D02E0E88
:1075B000F66E170EF76E00012FEC0CF002010C6B4B
:1075C0000C51095D3BE3320EF66E170EF76E0B0E93
:1075D0000A01E16F0001B1EC0CF00CC2E1FA570EA8
:1075E0000A01E26F0001C6EC0CF03D0E9EA8FED72A
:1075F000AD6E200E9EA8FED7AD6E036A02010C513F
:10760000FE0FE96E060E0320EA6EEFCF44F844C881
:10761000E1FA570E0A01E26F0001C6EC0CF0200EF1
:107620009EA8FED7AD6E0A0E9EA8FED7AD6E0D0EBB
:107630009EA8FED7AD6E02010C2BC2D7440EF66E8B
:10764000170EF76E0B0E0A01E16F0001B1EC0CF0A2
:107650000FC2E1FA570E0A01E26F0001C6EC0CF00E
:10766000200E9EA8FED7AD6E0A0E9EA8FED7AD6E68
:107670000D0E9EA8FED7AD6E02016D6B6C6B6B6B31
:10768000010E6A6F0B0E106F0001000C150E0A013F
:10769000ED6F0001B3EC0DF07EC2EDFAB3EC0DF02E
:1076A00002018651060DF3507E250801516F000E30
:1076B00002017F210801526F51C8EDFA0001B3ECBD
:1076C0000DF0750E0A01ED6F0001B3EC0DF080C2F4
:1076D000EDFAB3EC0DF002018751080DF35080254F
:1076E0000801516F000E020181210801526F010E45
:1076F000515F000E525B51C8EDFA0001B3EC0DF082
:107700000801456B45510608D8B41DD1476B0201ED
:1077100086510801475DD8B414D1466B465108081C
:10772000D8B40DD1442D14D04551080DF350462541
:10773000006ED89000360050036A0001C1EC01F0E1
:107740000900F5CF03F00801496F03C04AF8A0D043
:107750004451020814E14551080DF3504625006ECE
:10776000D89000360050036A0001F9EC01F00900DE
:10777000F5CF03F00801496F03C04AF889D044519E
:10778000030814E14551080DF3504625006ED890CA
:1077900000360050036A000131EC02F00900F5CF19
:1077A00003F00801496F03C04AF872D0445104083D
:1077B00014E14551080DF3504625006ED89000366F
:1077C0000050036A000169EC02F00900F5CF03F0F4
:1077D0000801496F03C04AF85BD04451050814E121
:1077E0004551080DF3504625006ED89000360050E4
:1077F000036A0001A1EC02F00900F5CF03F00801D3
:10780000496F03C04AF844D04451060814E1455179
:10781000080DF3504625006ED89000360050036ADC
:107820000001D9EC02F00900F5CF03F00801496F1F
:1078300003C04AF82DD04451070814E14551080D02
:10784000F3504625006ED89000360050036A0001C0
:1078500011EC03F00900F5CF03F00801496F03C0F4
:107860004AF816D04451080813E14551080DF35069
:107870004625006ED89000360050036A000149EC9E
:1078800003F00900F5CF03F00801496F03C04AF87F
:1078900049510F0B516F526B51354F6F5235506F2D
:1078A0004F375037FC0E4F174A3349334A33493369
:1078B0004A3349334A3349330F0E4A1749510F0BA4
:1078C000516F526B51354D6F52354E6F4D374E37AC
:1078D000FC0E4D174A3349334A3349334A3349334F
:1078E0004A3349330F0E4A1749510F0B516F526BF0
:1078F00051354B6F52354C6F4B374C37FC0E4B1795
:107900004A3349334A3349334A3349334A33493393
:107910000F0E4A17486B020187510801485D0CE0C1
:107920004BC8F4FA4DC8F5FA4FC8F6FA0001CCEC92
:107930000FF00801482BEFD7010E4627EFD6472B53
:10794000E6D6452BDFD602018651060DF3507E2781
:10795000000E7F23010E876F866F0001000C02016D
:1079600008A956D081B03BD0880EF66E160EF76E81
:1079700000012FEC0CF0020108998A8A898C640EB0
:107980000801456F00017AEC11F08D90640E08013A
:10799000456F00017AEC11F00B0E936E0201856BBE
:1079A000846B0F0E836FFF0E826F010E876F866FE1
:1079B000060E0801436F00018FEC11F0070E08015D
:1079C000436F00018FEC11F089EC0EF072DD0201C3
:1079D000106B070E0801436F00018FEC11F03C0E95
:1079E0000A01DE6F180EDF6F0001C2EC0EF084A2F8
:1079F00007D02A0E0A01EA6F00012AEC11F006D026
:107A0000200E0A01EA6F00012AEC11F096D0020163
:107A100008B993D081A091D0A40EF66E160EF76E21
:107A200000012FEC0CF0020108898A948A988A9A46
:107A3000020E0801436F960E456F00017AEC11F0BB
:107A40000801432FF8D7898C020E436F960E456FBD
:107A500000017AEC11F00801432FF8D73F0E936E26
:107A6000020E436FFA0E456F00017AEC11F0080127
:107A7000432FF8D7BE0EF66E160EF76E00012FECF0
:107A80000CF08D8084B401D0FDD7899CD00EF66EA9
:107A9000160EF76E2FEC0CF089EC0EF00A01DE6B7F
:107AA000DF6B0001C2EC0EF0020E0201876F866FE1
:107AB000856B0F0E846F836FFF0E826FE20EF66E82
:107AC000160EF76E00016AEC11F02A0E0A01DE6F45
:107AD000180EDF6F0001C2EC0EF0010E0201876F7D
:107AE000866F856B846B0F0E836FFF0E826F070EA0
:107AF0000801446F0001CADD300E0A01DE6F180E66
:107B0000DF6F0001C2EC0EF0010E0201876F866F7D
:107B1000856B846B0F0E836FFF0E826F080E08015A
:107B2000446F0001B3DD010E0201876F866F856B24
:107B3000846B0F0E836FFF0E826F0001000C0C0E22
:107B4000016EC250C30B0110C26EC282C2B2FED718
:107B5000C4CF45F80801C3CF44F8455102081EE3DD
:107B600003E14451E3081AE3120E0A01DE6F250E09
:107B7000DF6F0001C2EC0EF00F0E0201856F846B07
:107B8000836FFF0E826F010E876F866F4E0EF66E4B
:107B9000180EF76E00016AEC11F008010001000CEC
:107BA0000A018E6B2AC80BFD29C80AFD28C809FDE9
:107BB00027C808FD080E0D010D6F8E0E0C6F000119
:107BC00097EC15F00A018F6B8F51F90833E38E0E95
:107BD0008F25E96E080EEA6ED8B0EA2AEF501F082A
:107BE00022E209D08E0E8F25E96E080EEA6ED8B01B
:107BF000EA2A00A018D0036A8E5108018C25016E74
:107C00008D5103220A018E0E8F25E96E080EEA6E51
:107C1000D8B0EA2AEFCF92FA03C0EAFF01C0E9FF29
:107C200092CAEFFF8E2B8E51F80802E2FA0E8F6F88
:107C30008F2BCAD78E51F9080DE3036A8E510801C4
:107C40008C25E96E8D510320EA6E200EEF6E0A013D
:107C50008E2BF0D700016CEF43F0AAC803F00801A7
:107C6000A9C8E9FFAAC8EAFFEF5239E0AAC8AEF8EE
:107C7000A9C8ADF8ACC8B0F8ABC8AFF8B0C803F04D
:107C8000AFC8E9FFB0C8EAFFEF5216E0ADC8E9FFA0
:107C9000AEC8EAFFEFCFB1F8B0C803F0AFC8E9FF54
:107CA000B0C8EAFFEF50B15D07E1AD2BD8B4AE2B01
:107CB000AF2BD8B4B02BE2D7B0C803F0AFC8E9FF00
:107CC000B0C8EAFFEF5205E1A9C801F0AAC802F066
:107CD00009D0A92BD8B4AA2B0001BFD70801000EE8
:107CE000016E026E0001000C0A01E26B1F0EE16FD3
:107CF0000001C6EC1FF001C01AF10801AA6B1F0EAB
:107D0000A96F010EAC6F860EAB6F0001A6DF01C03C
:107D100037F10801AA6B1F0EA96F010EAC6F810E1F
:107D2000AB6F00019ADF01C036F10801AA6B1F0E8C
:107D3000A96F010EAC6F950EAB6F00018EDF01C015
:107D400034F10801AA6B1F0EA96F010EAC6F8B0EE8
:107D5000AB6F000182DF01C033F10801AA6B1F0E77
:107D6000A96F010EAC6F900EAB6F000176DF01C002
:107D700039F10801AA6B1F0EA96F010EAC6F9A0EA4
:107D8000AB6F00016ADF01C035F10801AA6B1F0E5D
:107D9000A96F010EAC6F9F0EAB6F00015EDF01C0DB
:107DA00038F10801AA6B1F0EA96F010EAC6FA40E6B
:107DB000AB6F000152DF01C03AF10801AA6B1F0E40
:107DC000A96F010EAC6FA90EAB6F000146DF01C0B9
:107DD0003BF10801AA6B1F0EA96F010EAC6FAE0E2E
:107DE000AB6F00013ADF01C03CF10801AA6B1F0E26
:107DF000A96F010EAC6FB30EAB6F00012EDF01C097
:107E00003DF10801AA6B1F0EA96F010EAC6FB80EF1
:107E1000AB6F000122DF01C03EF1010137511A5D55
:107E20001C6F1A511C5DD8B41C6B36511A5D1B6F48
:107E30001A511B5DD8B41B6B34511A5D1E6F1A5159
:107E40001E5DD8B41E6B33511A5D1D6F1A511D5D36
:107E5000D8B41D6B39511A5D216F1A51215DD8B408
:107E6000216B35511A5D1F6F1A511F5DD8B41F6BFE
:107E700038511A5D206F1A51205DD8B4206B3A51E9
:107E80001A5D226F1A51225DD8B4226B3B511A5DE4
:107E9000236F1A51235DD8B4236B3C511A5D246FB4
:107EA0001A51245DD8B4246B3D511A5D256F1A51C7
:107EB000255DD8B4256B3E511A5D266F1A51265D9B
:107EC000D8B4266B1CC18CF81BC18DF81EC18EF86E
:107ED0001DC18FF821C190F81FC191F820C192F8FF
:107EE00022C193F823C194F824C195F825C196F8CE
:107EF00026C197F81B0E375D2B6F1B0E365D2A6F60
:107F00001B0E345D286F1B0E335D276F1B0E395D12
:107F10002D6F1B0E355D296F1B0E385D2C6F1B0EF0
:107F20003A5D2E6F1B0E3D5D316F1B0E3E5D326F55
:107F30000801A46BA56BA53D01D022D0A66BA6516C
:107F40000B0816E3036AA6518C0FE96E080E032096
:107F5000EA6EA551EF5C0AE1036AA451980FE96E3D
:107F6000080E0320EA6EA6C8EFFFA42BA62BE7D7C6
:107F7000A4510C0803E1FF0EA56F02D0A52BDBD79F
:107F80000B0EA76FA75325E0036AA751980FE96E60
:107F9000080E0320EA6EEF521AE1A753D8A4A707F0
:107FA000A7C8A4F8036AA451980FE96E080E03202D
:107FB000EA6EEFCFA8F8036AA8518C0FE96E080E9D
:107FC0000320EA6EEF5001011C5F03D00801A707F0
:107FD000D9D70B0E0801A76FA75325E0036AA75155
:107FE000980FE96E080E0320EA6EEF2C1AD0A75303
:107FF000D8A4A707A7C8A4F8036AA451980FE96EEC
:10800000080E0320EA6EEFCFA8F8036AA8518C0F80
:10801000E96E080E0320EA6EEF5001011B5F04D0E9
:108020000801A707D9D70101040E1C5F1B5F1C5173
:108030001F0802E2200E1C6F1B511F0802E2200ED7
:108040001B6F00016EEF43F008018E6B8D6B010119
:108050001B511F0858E21F0E2A2508018F6F906BD5
:10806000D8B0902B010E0A01E26F600EE16F90C84C
:10807000E4FA8FC8E3FAE66B1BC1E5FA0001E3EC12
:108080001FF01F0E08018C6F8C51010814E2036A67
:108090008C51600FE96E010E0320EA6EEF5020084C
:1080A00005E0010E01011B5F03D0080104D00101AE
:1080B00008018C07E9D71F0E8C6F8C51010814E260
:1080C000036A8C51600FE96E010E0320EA6EEF50D7
:1080D000200805E1010E01011B5F03D0080104D057
:1080E000010108018C07E9D7010EEA6E600EE96E06
:1080F000000E0001AAEC03F00A000900F550EE6E34
:108100000009FBE101011B51100827E3100ED88084
:108110001B55006ED89000320050600F08018F6F21
:10812000010E906FD8B0902B1F0E01012A25080177
:10813000916F926BD8B0922B90C8E2FA8FC8E1FA97
:1081400092C8E4FAE8CFE3FA0A01E66B1BC1E5FA4C
:108150000001E3EC1FF07BD001011B511F08D8A0E8
:1081600077D01F0E2A2508018F6F906BD8B0902B07
:10817000010E0A01E26F600EE16F90C8E4FA8FC849
:10818000E3FAE66B1BC1E5FA0001E3EC1FF0100E09
:1081900008018C6F8C51010810E2036A8C51600F4A
:1081A000E96E010E0320EA6EEF50200804E18CC84E
:1081B0008EF8010E8C6F8C07EDD78E5101011B5D7F
:1081C00008018D6F8D51100802E2100E8D6F010EA7
:1081D000EA6E600EE96E000E0001AAEC03F00A00E0
:1081E0000900F550EE6E0009FBE11F0E01012A2582
:1081F00008018F6F906BD8B0902B010E0A01E26FCF
:10820000600EE16F90C8E4FA8FC8E3FAE66B8EC89F
:10821000E5FA0001E3EC1FF01F0E01012A25080119
:108220008F6F906BD8B0902B8E518F27000E9023BC
:10823000010E0A01E26F700EE16F90C8E4FA8FC878
:10824000E3FAE66B8DC8E5FA0001E3EC1FF00101EB
:108250002A51E00812E2010E0A01E26F600EE16F9E
:10826000070EE46F750EE36FE66BAEC7E5FA00012B
:10827000E3EC1FF00201306B03D0010E0201306FFE
:1082800008018E6B8D6B01011C511F08D8B06DD099
:108290001F0E2B2508018F6F906BD8B0902B010E0D
:1082A0000A01E26F3F0EE16F90C8E4FA8FC8E3FA6B
:1082B000E66B1CC1E5FA0001E3EC1FF01F0E08019C
:1082C0008C6F8C51010814E2036A8C513F0FE96EE8
:1082D000010E0320EA6EEF50200805E0010E0101B7
:1082E0001C5F03D0080104D0010108018C07E9D705
:1082F0001F0E8C6F8C51010814E2036A8C513F0FE2
:10830000E96E010E0320EA6EEF50200805E1010E30
:1083100001011C5F03D0080104D0010108018C0792
:10832000E9D7200E8C6F8C51010810E2036A8C5142
:108330003F0FE96E010E0320EA6EEF50200804E1C2
:108340008CC88EF8010E8C6F8C07EDD7010EEA6E8B
:108350003F0EE96E000E0001AAEC03F00A000900CE
:10836000F550EE6E0009FBE101011C51100827E3F6
:10837000100ED8801C55006ED890003200503F0F70
:1083800008018F6F010E906FD8B0902B1F0E010166
:108390002B250801916F926BD8B0922B90C8E2FA0E
:1083A0008FC8E1FA92C8E4FAE8CFE3FA0A01E66B73
:1083B0001CC1E5FA0001E3EC1FF07BD001011C5168
:1083C0001F08D8A077D01F0E2B2508018F6F906B48
:1083D000D8B0902B010E0A01E26F3F0EE16F90C8FA
:1083E000E4FA8FC8E3FAE66B1CC1E5FA0001E3EC9E
:1083F0001FF0100E08018C6F8C51010810E2036A07
:108400008C513F0FE96E010E0320EA6EEF502008F9
:1084100004E18CC88EF8010E8C6F8C07EDD78E515D
:1084200001011C5D08018D6F8D51100802E2100ED4
:108430008D6F010EEA6E3F0EE96E000E0001AAEC90
:1084400003F00A000900F550EE6E0009FBE11F0E73
:1084500001012B2508018F6F906BD8B0902B010E76
:108460000A01E26F3F0EE16F90C8E4FA8FC8E3FAA9
:10847000E66B8EC8E5FA0001E3EC1FF01F0E010168
:108480002B2508018F6F906BD8B0902B8E518F27C2
:10849000000E9023010E0A01E26F4F0EE16F90C8AB
:1084A000E4FA8FC8E3FAE66B8DC8E5FA0001E3EC65
:1084B0001FF001012B51E0080FE2010EEA6E3F0EA2
:1084C000E96E000E000181EC03F00A000900F5508E
:1084D000EE6E0009FBE1010100016FEF43F0010EB8
:1084E000EA6E810EE96E000EC3EC03F00A0009008B
:1084F000F550EE6E0009FBE1010EEA6E860EE96EA4
:10850000000ECEEC03F00A000900F550EE6E0009F3
:10851000FBE1010EEA6E8B0EE96E000ED9EC03F062
:108520000A000900F550EE6E0009FBE1010EEA6E4B
:10853000900EE96E000EE4EC03F00A000900F5501D
:10854000EE6E0009FBE1010EEA6E950EE96E000E7B
:10855000EFEC03F00A000900F550EE6E0009FBE1B4
:10856000010EEA6E9A0EE96E000EFAEC03F00A00B4
:108570000900F550EE6E0009FBE1010EEA6E9F0E58
:10858000E96E000E05EC04F00A000900F550EE6EED
:108590000009FBE1010EEA6EA40EE96E000E10EC7C
:1085A00004F00A000900F550EE6E0009FBE1010E2F
:1085B000EA6EA90EE96E000E1BEC04F00A00090039
:1085C000F550EE6E0009FBE1010EEA6EAE0EE96EAB
:1085D000000E26EC04F00A000900F550EE6E0009CA
:1085E000FBE1010EEA6EB30EE96E000E31EC04F011
:1085F0000A000900F550EE6E0009FBE1010EEA6E7B
:10860000B80EE96E000E3CEC04F00A000900F550CB
:10861000EE6E0009FBE1EA6A1F0EE96E000E81ECC6
:1086200003F00A000900F550EE6E0009FBE1010EAF
:10863000EA6E600EE96E000EAAEC03F00A00090073
:10864000F550EE6E0009FBE1010EEA6E3F0EE96E99
:10865000000EAAEC03F00A000900F550EE6E0009C6
:10866000FBE1080EEA6E480EE96E000E47EC04F0DE
:108670000A000900F550EE6E0009FBE1080EEA6EF3
:10868000590EE96E000E47EC04F00A000900F5509F
:10869000EE6E0009FBE1080EEA6E6A0EE96E000E4E
:1086A00047EC04F00A000900F550EE6E0009FBE10A
:1086B000080EEA6E7B0EE96E000E47EC04F00A002D
:1086C0000900F550EE6E0009FBE108018D6B1F0EED
:1086D0008C6F0001D0EF3DF074EF3EF0B5D4080E82
:1086E0000A01E26F6A0EE16F010EE46F3F0EE36F65
:1086F000E66B100EE56F0001E3EC1FF008017A6BEA
:10870000080E0A01E26F7B0EE16F010EE46F4F0E5F
:10871000E36FE66B100EE56F0001E3EC1FF008015C
:108720008B6B080E0A01E26F480EE16F010EE46FD9
:10873000600EE36FE66B100EE56F0001E3EC1FF0D7
:108740000801586B080E0A01E26F590EE16F010E25
:10875000E46F700EE36FE66B100EE56F0001E3EC63
:108760001FF00801696B01011C51100819E3020E8A
:108770000201876F010E866F856B846B0F0E836F0E
:10878000F00E826F0A01DE6BDF6B0001C2EC0EF0AF
:10879000080EEA6E6A0EE96E8CEC28F024D0010116
:1087A000010E0201876F866F856B846B0F0E836FDE
:1087B000F00E826F0A01DE6BDF6B0001C2EC0EF07F
:1087C000080EEA6E6A0EE96E8CEC28F00A01DE6B88
:1087D000080EDF6F0001C2EC0EF0080EEA6E7B0E91
:1087E000E96E8CEC28F001011B51100819E3020E10
:1087F0000201876F010E866F856B846B836BFF0EA2
:10880000826F0A01DE6B100EDF6F0001C2EC0EF00A
:10881000080EEA6E480EE96E8CEC28F024D00101B7
:10882000010E0201876F866F856B846B836BFF0E71
:10883000826F0A01DE6B100EDF6F0001C2EC0EF0DA
:10884000080EEA6E480EE96E8CEC28F00A01DE6B29
:10885000180EDF6F0001C2EC0EF0080EEA6E590E22
:10886000E96E8CEC28F0010E0201876F866F856B34
:10887000846B0F0E836FFF0E826F0801146B156BF4
:10888000000152EF53F00801266B256B246B236B1C
:108890004BC70BFD4AC70AFD49C709FD48C708FD7C
:1088A000080E0D010D6F480E0C6F000197EC15F0CE
:1088B00008011E6B1D6B1C6B50C81BF8226B216BD3
:1088C000206B51C81FF81B371C371D371E371B374D
:1088D0001C371D371E371B371C371D371E371B37FC
:1088E0001C371D371E371B371C371D371E371B37EC
:1088F0001C371D371E371B371C371D371E37800EA0
:108900001B171EC826F81DC825F81CC824F81BC84C
:1089100023F81F512327205124232151252322519D
:1089200026230A0E2327000E242325232623180E90
:10893000F66E140EF76E0A0E0A01E16F0001B1EC3B
:108940000CF026C8E1FA570E0A01E26F0001C6ECEE
:108950000CF025C8E1FA570E0A01E26F0001C6ECDF
:108960000CF024C8E1FA570E0A01E26F0001C6ECD0
:108970000CF023C8E1FA570E0A01E26F0001C6ECC1
:108980000CF0200E9EA8FED7AD6E0A0E9EA8FED754
:10899000AD6E0D0E9EA8FED7AD6E25EF45F00A0117
:1089A000486B020E08012327000E242325232623CB
:1089B00026530AE1255308E12451010810E2FF0A79
:1089C00003E1235100080BE20A01482B000E0801C5
:1089D000235F020E245B000E255B265BE9D70A01AC
:1089E0004851070148250A01496F000E0701492136
:1089F0000A014A6F000E07014A210A014B6F000E5F
:108A000007014B210A014C6FE8CF0BFD4BCA0AFD51
:108A10004ACA09FD49CA08FD080E0D010D6F480E2E
:108A20000C6F000197EC15F00801166B480E23251A
:108A3000E96E080E2421EA6EEFCF16F8163B0F0EF2
:108A40001617000126EF45F01ED7A9D7E80EF66EDF
:108A5000130EF76E060E0A01E16F0001B1EC0CF087
:108A600016C8E1FA570E0A01E26F0001C6EC0CF0DD
:108A7000200E9EA8FED7AD6E0A0E9EA8FED7AD6E44
:108A80000D0E9EA8FED7AD6E08013A6B396B386BA0
:108A9000376B1651090807E13A6B010E396FF40E76
:108AA000386F376B5AD016510A0807E13A6B020E3D
:108AB000396F710E386F376B50D016510B0807E1C4
:108AC0003A6B020E396FEE0E386F376B46D0165187
:108AD000070807E13A6B010E396F770E386F376B75
:108AE0003CD016510C0807E13A6B030E396F6B0E40
:108AF000386F376B32D016510D0807E13A6B030E11
:108B0000396FE80E386F376B28D016510E0807E121
:108B10003A6B040E396FE20E386F376B1ED0165366
:108B200008E13A6B030E396F0D0E386F400E376F48
:108B300014D01651080808E13A6B010E396FB50ED2
:108B4000386F800E376F09D016510F0806E13A6B67
:108B5000396B030E386FE80E376FF60EF66E130E94
:108B6000F76E0A0E0A01E16F0001B1EC0CF03AC891
:108B7000E1FA570E0A01E26F0001C6EC0CF039C8A9
:108B8000E1FA570E0A01E26F0001C6EC0CF038C89A
:108B9000E1FA570E0A01E26F0001C6EC0CF037C88B
:108BA000E1FA570E0A01E26F0001C6EC0CF0200E4C
:108BB0009EA8FED7AD6E0A0E9EA8FED7AD6E0D0E16
:108BC0009EA8FED7AD6E08013A31036E3931026EB0
:108BD0003831016E3731006E033202320132003219
:108BE00003320232013200321F0E031603C04BF86B
:108BF00002C04AF801C049F800C048F8D8922EC80F
:108C0000F0FA2DC8EFFA2CC8EEFA2BC8EDFA03C023
:108C1000F4FA02C0F3FA01C0F2FA00C0F1FA00015E
:108C20005AEC16F003C036F802C035F801C034F82B
:108C300000C033F8080EF66E140EF76E0A0E0A0125
:108C4000E16F0001B1EC0CF036C8E1FA570E0A01F1
:108C5000E26F0001C6EC0CF035C8E1FA570E0A01CC
:108C6000E26F0001C6EC0CF034C8E1FA570E0A01BD
:108C7000E26F0001C6EC0CF033C8E1FA570E0A01AE
:108C8000E26F0001C6EC0CF0200E9EA8FED7AD6E80
:108C90005CEF53F00201079F2C0EF66E0D0EF76E7F
:108CA00000012FEC0CF0020131B7F6D0440EF66E45
:108CB0000D0EF76E00012FEC0CF0E0C653FADFC684
:108CC00052FADEC651FADDC650FA0A015F6B0601A0
:108CD000B1510A0151254C6F0601B2510A015221CE
:108CE0004D6F0601B3510A0153214E6F0601B45175
:108CF0000A015F214F6F4FCA0BFD4ECA0AFD4DCAD4
:108D000009FD4CCA08FD080E0D010D6F480E0C6FD1
:108D1000000197EC15F00A015F6B006A0050505D8E
:108D20005C6F515151595D6F525152595E6F5351A1
:108D300053595F6FD8905C35586F5D35596F5E350C
:108D40005A6F5F355B6F5BCA4BFA5ACA4AFA59CA07
:108D500049FA58CA48FA4B53D8A49BD04A53D8A4CE
:108D600098D049510108D8A094D004E14851FE0898
:108D7000D8A08FD0010E48255C6F000E49215D6F91
:108D8000000E4A21000E4B21480E5C25E96E080EAC
:108D90005D21EA6EEFCF44F808010A01576B566B6C
:108DA000556B44C854FA56CA57FA55CA56FA54CAAB
:108DB00055FA546B480E4825E96E080E4921EA6EB3
:108DC000EFCF45F8080145510A015427000E5523FD
:108DD0005623572357530AE1565308E15551FE08CD
:108DE00008E2FF0A03E15451EF0803E2000E016EAE
:108DF000F0D1010E5025006E000E5121016E000EC3
:108E00005221026E000E5321036E0050545D09E1A1
:108E10000150555D06E10250565D03E10350575D78
:108E200029E00201078F07A721D0000E07BF010E1E
:108E30000A015C6F4E0EF66E0D0EF76E080EE16FB6
:108E40000001B1EC0CF05CCAE1FA570E0A01E26FC6
:108E50000001C6EC0CF0580EF66E0D0EF76E040E07
:108E60000A01E16F0001B1EC0CF00201010E016E8C
:108E70000A01AFD157CA53FA56CA52FA55CA51FA23
:108E800054CA50FA020E4827000E49234A234B23A6
:108E900062D71CD79ED1020131A79CD15E0EF66E1F
:108EA0000D0EF76E00012FEC0CF0E0C653FADFC692
:108EB00052FADEC651FADDC650FA0A0153315F6F2D
:108EC00052315E6F51315D6F50315C6F5F335E3395
:108ED0005D335C335F335E335D335C335F335E330E
:108EE0005D335C335F335E335D335C335F335E33FE
:108EF0005D335C335F335E335D335C33010E5F178C
:108F00000601B1510A015C254C6F0601B2510A01FC
:108F10005D214D6F0601B3510A015E214E6F0601BE
:108F2000B4510A015F214F6F4FCA0BFD4ECA0AFDB3
:108F30004DCA09FD4CCA08FD080E0D010D6F480E03
:108F40000C6F000197EC15F00A0153315F6F52313D
:108F50005E6F51315D6F50315C6F5F335E335D33F7
:108F60005C335F335E335D335C335F335E335D337D
:108F70005C335F335E335D335C335F335E335D336D
:108F80005C335F335E335D335C33010E5F175C35FA
:108F9000006E5D35016E5E35026E5F35036E003624
:108FA0000136023603360036013602360336003605
:108FB00001360236033600360136023603360036F5
:108FC0000136023603360036013602360336800E8D
:108FD00000160050505D5C6F015051595D6F02509A
:108FE00052595E6F035053595F6F5C35586F5D3552
:108FF000596F5E355A6F5F355B6F583759375A373F
:109000005B37FC0E58175BCA4BFA5ACA4AFA59CA60
:1090100049FA58CA48FA4B53D8A4DAD04A53D8A4CC
:10902000D7D049510108D8A0D3D004E14851FC0859
:10903000D8A0CED0030E48255C6F000E49215D6F8D
:10904000000E4A21000E4B21480E5C25E96E080EE9
:109050005D21EA6EEFCF44F808010A01576B566BA9
:10906000556B44C854FA56CA57FA55CA56FA54CAE8
:1090700055FA546B020E48255C6F000E49215D6F56
:10908000000E4A21000E4B21480E5C25E96E080EA9
:109090005D21EA6EEFCF45F8080145510A015427DA
:1090A000000E55235623572356CA57FA55CA56FA67
:1090B00054CA55FA546B010E48255C6F000E4921C5
:1090C0005D6F000E4A21000E4B21480E5C25E96EB3
:1090D000080E5D21EA6EEFCF46F8080146510A01FD
:1090E0005427000E55235623572356CA57FA55CAFC
:1090F00056FA54CA55FA546B480E4825E96E080EC4
:109100004921EA6EEFCF47F8080147510A01542779
:10911000000E552356235723543D0AD0553D08D001
:10912000563D06D057510F0803E1000E016E51D095
:10913000010E5025006E000E5121016E000E5221CD
:10914000026E000E5321036E0050545D09E1015080
:10915000555D06E10250565D03E10350575D29E07D
:109160000201078F07A721D0000E07BF010E0A01D9
:109170005C6F680EF66E0D0EF76E080EE16F000163
:10918000B1EC0CF05CCAE1FA570E0A01E26F000183
:10919000C6EC0CF0720EF66E0D0EF76E040E0A01A0
:1091A000E16F0001B1EC0CF00201010E016E0A0149
:1091B00010D057CA53FA56CA52FA55CA51FA54CA6D
:1091C00050FA040E4827000E49234A234B2323D785
:1091D00075D602010001C7EF54F00A01DE6B250EBF
:1091E000DF6F0001C2EC0EF0010E0201876F866F87
:1091F000856B846B0F0E836FA00E826F132D09D0C9
:10920000560EF66E180EF76E00016AEC11F00AD0D9
:109210000201135307E1580EF66E180EF76E0001A7
:109220006AEC11F0060E0A01DE6F250EDF6F0001F9
:10923000C2EC0EF0010E0201876F866F122D09D06D
:109240005A0EF66E180EF76E00016AEC11F00AD095
:109250000201125308E15C0EF66E180EF76E000163
:109260006AEC11F002010001000C0201319931B7E2
:109270001FD0D8900601ED35006EEE35016EEF354A
:10928000026EF035036E0050C1250801446F015095
:109290000601C2210801456F02500601C3210801E1
:1092A000466F03500601C4210801476F25D0020113
:1092B00031A723D00601ED35006EEE35016EEF3596
:1092C000026EF035036E0036013602360336FC0EB0
:1092D00000160050C1250801446F01500601C2214B
:1092E0000801456F02500601C3210801466F035073
:1092F0000601C4210801476F020107A52FD0780E8F
:10930000F66E0D0EF76E140E0A01E16F0001B1EC5E
:109310000CF0F4C6E1FA570E0A01E26F0001C6EC48
:109320000CF0F3C6E1FA570E0A01E26F0001C6EC39
:109330000CF0F2C6E1FA570E0A01E26F0001C6EC2A
:109340000CF0F1C6E1FA570E0A01E26F0001C6EC1B
:109350000CF0200E9EA8FED7AD6E020107A52FD0FF
:10936000920EF66E0D0EF76E0A0E0A01E16F000105
:10937000B1EC0CF047C8E1FA570E0A01E26F0001A8
:10938000C6EC0CF046C8E1FA570E0A01E26F000184
:10939000C6EC0CF045C8E1FA570E0A01E26F000175
:1093A000C6EC0CF044C8E1FA570E0A01E26F000166
:1093B000C6EC0CF0200E9EA8FED7AD6E020107AFE2
:1093C000F7D107A508D0A20EF66E0D0EF76E0001BC
:1093D0002FEC0CF0020131B7ABD00601FD531CE1BC
:1093E000010E080144254C6F000E45214D6F000E03
:1093F00046214E6F000E47214F6FE8CFEAFA4EC864
:10940000E9FA4DC8E8FA4CC8E7FA00011AEC1EF078
:1094100000C048F81DD00601FD2D1BD0010E08012B
:1094200044254C6F000E45214D6F000E46214E6FB6
:10943000000E47214F6FE8CFEAFA4EC8E9FA4DC84F
:10944000E8FA4CC8E7FA00018CEC1EF001C048F8BD
:109450000601F46BF36BF26B48C8F1F6F3C6F4F651
:10946000F2C6F3F6F1C6F2F6F16BFD530FE147C811
:10947000EAFA46C8E9FA45C8E8FA44C8E7FA00013A
:109480001AEC1EF000C049F810D00601FD2D0DD0D9
:1094900047C8EAFA46C8E9FA45C8E8FA44C8E7FA0C
:1094A00000018CEC1EF001C049F808014951060189
:1094B000F127000EF223F323F423F36BF46BF45340
:1094C0002FE1F3532DE1F251FF082AE303E1F151BB
:1094D000EF0826E3D890F135006EF235016EF335D2
:1094E000026EF435036E0050C1250801446F01502F
:1094F0000601C2210801456F02500601C32108017F
:10950000466F03500601C4210801476F010E070191
:109510004C27D8B04D2BD8B44E2BD8B44F2B06D0F7
:1095200002013189010E016E83D107013FD1020191
:1095300031A73BD10601FD531CE1030E0801442570
:109540004C6F000E45214D6F000E46214E6F000EF0
:1095500047214F6FE8CFEAFA4EC8E9FA4DC8E8FA5A
:109560004CC8E7FA00011AEC1EF000C048F81DD004
:109570000601FD2D1BD0030E080144254C6F000E83
:1095800045214D6F000E46214E6F000E47214F6F53
:10959000E8CFEAFA4EC8E9FA4DC8E8FA4CC8E7FA4B
:1095A00000018CEC1EF001C048F80601F46BF36B6F
:1095B000F26B48C8F1F6F3C6F4F6F2C6F3F6F1C65C
:1095C000F2F6F16BFD531CE1020E080144254C6FCD
:1095D000000E45214D6F000E46214E6F000E4721B3
:1095E0004F6FE8CFEAFA4EC8E9FA4DC8E8FA4CC81E
:1095F000E7FA00011AEC1EF000C049F81DD0060180
:10960000FD2D1AD0020E080144254C6F000E452195
:109610004D6F000E46214E6F000E47214F6FE8CF71
:10962000EAFA4EC8E9FA4DC8E8FA4CC8E7FA000170
:109630008CEC1EF001C049F8080149510601F127E0
:10964000000EF223F323F423F3C6F4F6F2C6F3F686
:10965000F1C6F2F6F16BFD531CE1010E0801442541
:109660004C6F000E45214D6F000E46214E6F000ECF
:1096700047214F6FE8CFEAFA4EC8E9FA4DC8E8FA39
:109680004CC8E7FA00011AEC1EF000C04AF81DD0E1
:109690000601FD2D1AD0010E080144254C6F000E65
:1096A00045214D6F000E46214E6F000E47214F6F32
:1096B000E8CFEAFA4EC8E9FA4DC8E8FA4CC8E7FA2A
:1096C00000018CEC1EF001C04AF808014A51060165
:1096D000F127000EF223F323F423F3C6F4F6F2C6C7
:1096E000F3F6F1C6F2F6F16BFD530FE147C8EAFA63
:1096F00046C8E9FA45C8E8FA44C8E7FA00011AEC96
:109700001EF000C04BF810D00601FD2D0DD047C84B
:10971000EAFA46C8E9FA45C8E8FA44C8E7FA000197
:109720008CEC1EF001C04BF808014B510601F127EB
:10973000000EF223F323F423F13D07D0F23D05D0D0
:10974000F33D03D0F4510F082BE0F135006EF235F4
:10975000016EF335026EF435036E003601360236C3
:109760000336FC0E00160050C1250801446F01505D
:109770000601C2210801456F02500601C3210801FC
:10978000466F03500601C4210801476F010E07010F
:109790004C27D8B04D2BD8B44E2BD8B44F2B06D075
:1097A00002013189010E016E43D007013ED0020152
:1097B00007BF3AD0010E0601ED25F16F000EEE2134
:1097C000F26F000EEF21F36F000EF021F46F010E27
:1097D00007014C27D8B04D2BD8B44E2BD8B44F2B03
:1097E0000801045107014C5D14E10801055107010E
:1097F0004D5D0FE10801065107014E5D0AE10801C8
:10980000075107014F5D05E102013189010E016E2B
:109810000FD0020107A508D0AC0EF66E0D0EF76E44
:1098200000012FEC0CF002010701000E016E020195
:10983000000140EF55F0020107A507D0B00EF66E0B
:10984000080EF76E00012FEC0CF0020E0801526FAB
:10985000536BCD0E546F040E556F000181EC0CF06C
:10986000020E0801526F536BCD0E546F040E556FEC
:10987000000181EC0CF0020E0801526F040E536FD0
:10988000546B556B000181EC0CF0000C0101BE51D2
:10989000BD5DFDE0036ABE51E50FE96E010E0320D8
:1098A000EA6EEFCF45F80801010E0101BE251F0B3E
:1098B000BE6F080145C801F00001ACEF4EF0AA6A86
:1098C000010EA96E37C2A8FFA69CA69EA684F250E0
:1098D000006EF29E0F01550EA76EAA0EA76EA6820D
:1098E000A6B2FED7A6940050F212AA6A020EA96E82
:1098F00012C2A8FFA69CA69EA684F2CF00F0F29EFC
:10990000550EA76EAA0EA76EA682A6B2FED7A69483
:109910000050F212AA6A030EA96E13C2A8FFA69CF9
:10992000A69EA684F2CF00F0F29E550EA76EAA0E58
:10993000A76EA682A6B2FED7A6940050F21200012E
:10994000000C7AC87DF879C87FF878C87EF80801DD
:109950007C5303E17B51000816E27FC803F07EC808
:10996000E9FF7FC8EAFF7D51EF5C05E17EC801F0A9
:109970007FC802F00BD07E2BD8B47F2B7B51D8B49C
:109980007C077B07E5D7000E016E026E0001000C1C
:1099900008017A517C19800B7E6F7AAF05D0791F50
:1099A0007A1F792BD8B47A2B7CAF05D07B1F7C1F14
:1099B0007B2BD8B47C2B79517B03F3CF01F0F4CF10
:1099C00000F07C03F35000267A517B03F350002013
:1099D000026E7EAF05D0011E021E012AD8B4022AF3
:1099E000000149EF4EF00801516B506B300E536F80
:1099F000310E546F320E556F330E566F340E576F53
:109A0000350E586F360E596F370E5A6F380E5B6F22
:109A1000390E5C6F610E5D6F620E5E6F630E5F6F7D
:109A2000640E606F650E616F660E626F670E636F26
:109A3000680E646F690E656F6A0E666F6B0E676FF6
:109A40006C0E686F6D0E696F6E0E6A6F6F0E6B6FC6
:109A5000700E6C6F710E6D6F730E6E6F740E6F6F94
:109A6000750E706F760E716F770E726F780E736F62
:109A7000790E746F7A0E756F766B46C84BF845C8D1
:109A80004AF84BC803F04AC8E9FF4BC8EAFFEF5059
:109A9000200804E14A2BD8B44B2BF3D74BC803F072
:109AA0004AC8E9FF4BC8EAFFEF502D0809E04BC850
:109AB00003F04AC8E9FF4BC8EAFFEF502B080BE15F
:109AC0004BC803F04A514A2BD8B44B2BE96E03C064
:109AD000EAFFEF5001D02B0E526F52512D080AE0D1
:109AE00049BF08D0492D01D005D049BF05D0495103
:109AF000240802E20DD184D049534CE049511008AA
:109B00001FE14BC803F04AC8E9FF4BC8EAFFEF501A
:109B1000300816E1010E4A25E96E000E4B21EA6E6F
:109B2000EF50780809E0010E4A25E96E000E4B213E
:109B3000EA6EEF50580804E1020E4A27000E4B234C
:109B4000495108080DE14BC803F04AC8E9FF4BC86A
:109B5000EAFFEF50300804E1010E4A27000E4B23C4
:109B60004951020816E14BC803F04AC8E9FF4BC847
:109B7000EAFFEF5030080DE1010E4A25E96E000EB4
:109B80004B21EA6EEF50620804E1020E4A27000EF4
:109B90004B2336D04BC803F04AC8E9FF4BC8EAFF55
:109BA000EF50300803E00A0E496F2AD0010E4A2513
:109BB000E96E000E4B21EA6EEF50780809E0010EC5
:109BC0004A25E96E000E4B21EA6EEF50580807E176
:109BD000100E496F020E4A27000E4B2311D0010EC2
:109BE0004A25E96E000E4B21EA6EEF50620806E14D
:109BF000020E496F4A27000E4B2302D0080E496F10
:109C00004BC84DF84AC84CF84BC803F04AC8E9FFA6
:109C10004BC8EAFFEF50300804E14A2BD8B44B2B75
:109C2000F3D74BC803F04AC8E9FF4BC8EAFFEFCFB0
:109C300077F87751400806E277515A0803E37751E5
:109C4000200901D07751776F080E796F530E786F26
:109C500077C87AF87C6B49C87BF8000172DE02C0D5
:109C60004FF801C04EF808014E5302E14F534AE04D
:109C7000036A4951006EE8BE0306776F03C078F8A7
:109C800051C87AF850C879F803C07CF87B6F00019E
:109C90007FD601C077F8530E08014E5D006E080EA6
:109CA0004F59036E00500124016E0250032201C07F
:109CB00050F803C051F84A2BD8B44B2B4BC803F0D3
:109CC0004AC8E9FF4BC8EAFFEFCF77F87751400861
:109CD00006E277515A0803E37751200901D0775102
:109CE000776F080E796F530E786F77C87AF87C6BB0
:109CF00049C87BF8000125DE02C04FF801C04EF8CC
:109D0000B2D708014A514C5D13E14B514D5D10E152
:109D10004751481109E047C8E9FF48C8EAFF46C86B
:109D2000ECFFED5245C8EFFF000E016E026E10D041
:109D30004751481109E047C8E9FF48C8EAFF4BC846
:109D4000ECFFED524AC8EFFF50C801F051C802F0D5
:109D5000000197EF4FF09AD501C0E0F10101E05109
:109D60002B0814E10201375110080EE23707020EEA
:109D70000801526F0B0E536F37C254F837C255F8B3
:109D8000000181EC0CF002019AD00101E0512D0894
:109D900014E10201373D01D00ED0372B020E08012D
:109DA000526F0B0E536F37C254F837C255F800018B
:109DB00081EC0CF0020183D00101E05162080EE158
:109DC000FF0E02011C27D8A01D27D8A01E27D8A04F
:109DD0001F27010E016ECED072D00101E0516E0836
:109DE0000EE1010E02011C27D8B01D2BD8B41E2B8A
:109DF000D8B41F2B010E016EBDD061D00101E0511E
:109E000068080DE1020107B308D0596B586B576B16
:109E1000640E566F020E016EADD051D00101E051BB
:109E200070080DE1020107A308D0596B586B576BFE
:109E3000640E566F020E016E9DD041D00101E051BB
:109E4000720807E10201125302E1010E126F37D0CE
:109E50000101E051610806E10201122D01D0126BEF
:109E60002ED00101E051630807E10201135302E122
:109E7000010E136F24D00101E051730806E10201C5
:109E8000132D01D0136B1BD00101E0510D0809E126
:109E9000036ADF51BF0FE96E010E0320EA6EEF6A1D
:109EA0000ED0036ADF51BF0FE96E010E0320EA6E88
:109EB000E0C1EFFFDF2B000E016E02015BD000015D
:109EC000FEDCEDEC48F0010E0A01E26FBF0EE16F1F
:109ED0000001C6EC1FF00150000849E23C0EF66E8E
:109EE000180EF76E0C0E0A01E16F0001B1EC0CF0D8
:109EF000010EEA6EBF0EE96E2CEC20F0200E9EA83B
:109F0000FED7AD6E0A0E9EA8FED7AD6E0D0E9EA8B2
:109F1000FED7AD6E010E0801466FBF0E456F080EED
:109F2000486F440E476F0A0E496F00015CD502C0AE
:109F300006F201C005F202011F6B1E6B06C21DF284
:109F400005C21CF2010EEA6EBF0EE96E000E0001A2
:109F500081EC03F00A000900F550EE6E0009FBE108
:109F60000101DF6B010E016E020104D00001000E41
:109F7000016E02010001000C0801516B506B83A8B7
:109F800001D0A9D1030E526F040E536F546B556B61
:109F9000000181EC0CF00801366B356B02C034F81F
:109FA00001C033F883A801D096D1D89236C8F0FA10
:109FB00035C8EFFA34C8EEFA33C8EDFA0A01F46B8B
:109FC000F36BF26B3C0EF16F00015AEC16F003C01C
:109FD00042F802C041F801C040F800C03FF842C852
:109FE000E4FA41C8E3FA40C8E2FA3FC8E1FA0A01DC
:109FF000E86BE76BE66B3C0EE56F00012CEC16F0AE
:10A0000000500801335D3B6F015034593C6F0250E2
:10A0100035593D6F035036593E6F83A801D05BD14F
:10A02000420E0A01DE6F300EDF6F0001C2EC0EF04F
:10A030000201856B846B836B0F0E826F020E876F3C
:10A04000010E866F3FC8DEFA0A01DF6F00019FEC48
:10A0500028F02A0EF66E140EF76E6AEC11F03BC86B
:10A06000DEFA010E0A01DF6F00019FEC28F0010EFD
:10A070000201876F866F83A803D008012CD10201EB
:10A0800083A802D0080127D1030E0801526F080EE1
:10A09000536F546B556B000181EC0CF002C051F80A
:10A0A00001C050F8080151C850F8516B513350337A
:10A0B0005133503351335033513350330F0E511706
:10A0C00083A801D008D14E0E0A01DE6F250EDF6F86
:10A0D0000001C2EC0EF00201856B846B0F0E836FE2
:10A0E000600E826F080150510E080BE1515309E1D7
:10A0F0002C0EF66E140EF76E00016AEC11F0BDD056
:10A10000080150510D080BE1515309E1300EF66E74
:10A11000140EF76E00016AEC11F0AFD00801505137
:10A120000C080BE1515309E1340EF66E140EF76E74
:10A1300000016AEC11F0A1D0080150510B080BE1AD
:10A14000515309E1380EF66E140EF76E00016AECF9
:10A1500011F093D0080150510A080BE1515309E165
:10A160003C0EF66E140EF76E00016AEC11F085D00D
:10A170000801505109080BE1515309E1400EF66EF8
:10A18000140EF76E00016AEC11F077D008015051FF
:10A1900008080BE1515309E1440EF66E140EF76EF8
:10A1A00000016AEC11F069D00801505107080BE179
:10A1B000515309E1480EF66E140EF76E00016AEC79
:10A1C00011F05BD00801505106080BE1515309E131
:10A1D0004C0EF66E140EF76E00016AEC11F04DD0C5
:10A1E0000801505105080BE1515309E1500EF66E7C
:10A1F000140EF76E00016AEC11F03FD008015051C7
:10A2000004080BE1515309E1540EF66E140EF76E7B
:10A2100000016AEC11F031D00801505103080BE144
:10A22000515309E1580EF66E140EF76E00016AECF8
:10A2300011F023D00801505102080BE1515309E1FC
:10A240005C0EF66E140EF76E00016AEC11F015D07C
:10A250000801502D0BD0515309E1600EF66E140E1B
:10A26000F76E00016AEC11F008D00801640EF66E7A
:10A27000140EF76E00016AEC11F083A802D00801F9
:10A280002AD00801145327E1155308E151C818F8E2
:10A2900050C817F851C81AF850C819F8152D04D02D
:10A2A00051C818F850C817F81551020804E151C8F0
:10A2B0001AF850C819F883A801D00DD0152B1551E4
:10A2C0000308D8B4156B1951175D03E11A51185DD5
:10A2D00002E0010E146F0001000C080144C84AF8A6
:10A2E00045C84BF846C844F847C845F8466B476B25
:10A2F00044C848F845C849F88A9AFF0E0D011E6FF8
:10A300000001BDEC11F0500E0D01166F186B176BAC
:10A31000020E1A6F196BFF0E1B6F0001E8EC11F0B3
:10A32000015202E00801E9D7FF0E0D011E6F000186
:10A33000BDEC11F0FF0E0D011E6F0001BDEC11F020
:10A340008A8A8A9A510E0D01166F49C818FD48C8AD
:10A3500017FD4BC81AFD4AC819FDFF0E1B6F0001FF
:10A3600075EC15F0FF0E0D011E6F0001BDEC11F034
:10A3700001C04FF808014F5302E00001F3D7FF0E70
:10A380000D011E6F0001BDEC11F00150FE0803E04D
:10A390000801F5D700018C968C948C86020131B9A6
:10A3A00030D008014D6B4D51100829E083B80BD017
:10A3B0003DC232F83CC231F83BC230F83AC22FF805
:10A3C0000001DADD080183B801D0FDD78A884C6B23
:10A3D0004C51200812E0070E4E6F4E3D01D00BD0BD
:10A3E0008A948A8481B602D08C9201D08C828C842B
:10A3F0008C944E07F2D74C2BEBD74D2BD4D75CD097
:10A40000020131A959D008014D6B4D51100854E09B
:10A4100083B80BD03DC232F83CC231F83BC230F8B1
:10A420003AC22FF80001A8DD080183B801D0FDD79A
:10A430008A884C6B4C5120083DE0070E4E6F4E3D14
:10A4400001D024D08A948A84070150530CE15153DF
:10A450000AE1525308E1535306E10201302D01D0C5
:10A460008C920FD00701505306E1515304E152532F
:10A4700002E1535305E081B602D08C9201D08C8268
:10A4800002018C848C9408014E07D9D707015053E0
:10A4900006E1515304E1525302E1535308E0FF0E29
:10A4A0005027D8A05127D8A05227D8A05327080159
:10A4B0004C2BC0D74D2BA9D7FF0E0D011E6F0001ED
:10A4C000BDEC11F08A8A000E016EE8EF57F0020130
:10A4D0001C530EE11D530CE11E530AE11F5308E10A
:10A4E00017C21FF216C21EF215C21DF214C21CF2D0
:10A4F00017511F5D11E30BE116511E5D0DE307E1DE
:10A5000015511D5D09E303E11C51145D05E21F6B4C
:10A510001E6B1D6B010E1C6F000189EC0EF0020119
:10A5200031A507D0AE0E0A01ED6F0001B3EC0DF0BE
:10A5300002010791596B586B576B566B079308B123
:10A5400008D0010E0801446F000195EC2AF009D0F3
:10A55000020108A106D0020E0801446F000195EC2B
:10A560002AF00601FD5311E1D8900201426B070168
:10A5700048350201436F070149350201446F070165
:10A580004A350201456F0CD00601FD2D08D04BC79E
:10A5900045F24AC744F249C743F248C742F20201B2
:10A5A00007A565D0560EF66E170EF76E0A0E0A0155
:10A5B000E16F0001B1EC0CF045C2E1FA570E0A015F
:10A5C000E26F0001C6EC0CF044C2E1FA570E0A013A
:10A5D000E26F0001C6EC0CF043C2E1FA570E0A012B
:10A5E000E26F0001C6EC0CF042C2E1FA570E0A011C
:10A5F000E26F0001C6EC0CF0200E9EA8FED7AD6EF7
:10A60000660EF66E170EF76E100E0A01E16F00016E
:10A61000B1EC0CF0ECC6E1FA570E0A01E26F000152
:10A62000C6EC0CF0EBC6E1FA570E0A01E26F00012E
:10A63000C6EC0CF0EAC6E1FA570E0A01E26F00011F
:10A64000C6EC0CF0E9C6E1FA570E0A01E26F000110
:10A65000C6EC0CF0200E9EA8FED7AD6E0A0E9EA88A
:10A66000FED7AD6E0D0E9EA8FED7AD6E02014BC794
:10A670002AF84AC729F849C728F848C727F8ECC676
:10A680002EF8EBC62DF8EAC62CF8E9C62BF81DC249
:10A6900045F81CC244F81DC247F81CC246F8000128
:10A6A0006FEF42F01DC245F81CC244F81DC247F8C6
:10A6B0001CC246F824EF45F0120E0A01DE6F300E80
:10A6C000DF6F0001C2EC0EF00201856B846B0F0E90
:10A6D000836FFF0E826F020E876F010E866F430E2F
:10A6E000E96E1FC2E1FA1EC2E0FA1DC2DFFA1CC207
:10A6F000DEFA0001E2EC28F02F0E0A01EA6F0001F9
:10A700002AEC11F0430EE96E17C2E1FA16C2E0FA24
:10A7100015C2DFFA14C2DEFAE2EC28F00801076B7A
:10A72000066B056B010E046FD890446B06019135E2
:10A730000801456F060192350801466F0601933501
:10A740000801476FE8CFE4FA46C8E3FA45C8E2FAE1
:10A7500044C8E1FA07C8E8FA06C8E7FA05C8E6FA05
:10A7600004C8E5FA00012CEC16F003500601EC5D7C
:10A7700017E30BE10250EB5D13E307E10150EA5DE3
:10A780000FE303E1E951005C0BE2010E080104272D
:10A79000D8B0052BD8B4062BD8B4072BC5D70601E3
:10A7A0007E0EF66E170EF76E170E0A01E16F0001AE
:10A7B000B1EC0CF007C8E1FA570E0A01E26F000194
:10A7C000C6EC0CF006C8E1FA570E0A01E26F000170
:10A7D000C6EC0CF005C8E1FA570E0A01E26F000161
:10A7E000C6EC0CF004C8E1FA570E0A01E26F000152
:10A7F000C6EC0CF0200E9EA8FED7AD6E0A0E9EA8E9
:10A80000FED7AD6E0D0E9EA8FED7AD6E9C0EF66EF9
:10A81000170EF76E110E0A01E16F0001B1EC0CF09A
:10A82000ECC6E1FA570E0A01E26F0001C6EC0CF02B
:10A83000EBC6E1FA570E0A01E26F0001C6EC0CF01C
:10A84000EAC6E1FA570E0A01E26F0001C6EC0CF00D
:10A85000E9C6E1FA570E0A01E26F0001C6EC0CF0FE
:10A86000200E9EA8FED7AD6E0A0E9EA8FED7AD6E36
:10A870000D0E9EA8FED7AD6E010E0801045D446F5B
:10A88000000E0559456F000E0659466F000E075918
:10A89000476FE8CFE4FA46C8E3FA45C8E2FA44C88D
:10A8A000E1FA94C6E8FA93C6E7FA92C6E6FA91C6C8
:10A8B000E5FA00012CEC16F003C047F802C046F898
:10A8C00001C045F800C044F8D890006A080144353A
:10A8D000016E4535026E4635036E00500601E95D96
:10A8E0000701506F01500601EA590701516F0250EC
:10A8F0000601EB590701526F03500601EC5907019D
:10A90000536FB40EF66E170EF76E0A0E0A01E16F62
:10A910000001B1EC0CF053C7E1FA570E0A01E26FE7
:10A920000001C6EC0CF052C7E1FA570E0A01E26FC3
:10A930000001C6EC0CF051C7E1FA570E0A01E26FB4
:10A940000001C6EC0CF050C7E1FA570E0A01E26FA5
:10A950000001C6EC0CF0200E9EA8FED7AD6E0A0ECC
:10A960009EA8FED7AD6E0D0E9EA8FED7AD6E070158
:10A970004F6B4E6B4D6B4C6BE0C6F0F6DFC6EFF6DF
:10A98000DEC6EEF6DDC6EDF600014AEF46F0C60E75
:10A99000F66E170EF76E060E0A01E16F0001B1ECBC
:10A9A0000CF0010EEA6E3F0EE96E2CEC20F0200E4A
:10A9B0009EA8FED7AD6E2D0E9EA8FED7AD6E200EC2
:10A9C0009EA8FED7AD6E010EEA6E600EE96E2CEC0D
:10A9D00020F0D30EF66E170EF76E070E0A01E16F28
:10A9E0000001B1EC0CF0020107A507D0DC0EF66EF9
:10A9F000170EF76E00012FEC0CF00A01DE6B300E23
:10AA0000DF6F0001C2EC0EF0020E0201876F866F4D
:10AA1000030E0801446F000146EC3BF0EDEC48F0FA
:10AA20000801366B356B346B336B020E526F0B0EB5
:10AA3000536F37C254F837C255F8000181EC0CF05F
:10AA400007014F510801075DD8A0E1D214E10701C9
:10AA50004E510801065DD8A0DAD20DE107014D5133
:10AA60000801055DD8A0D3D206E107014C510801C9
:10AA7000045DD8A0CCD200019FEC3DF035EF49F049
:10AA8000020E0601ED5D0801446F000E0601EE594D
:10AA90000801456F000E0601EF590801466F000ED0
:10AAA0000601F0590801476FE8CFE4FA46C8E3FA17
:10AAB00045C8E2FA44C8E1FA94C6E8FA93C6E7FA50
:10AAC00092C6E6FA91C6E5FA00012CEC16F003C036
:10AAD0005DF202C05CF201C05BF200C05AF20601F6
:10AAE000D55102015A270601D65102015B23060106
:10AAF000D75102015C230601D85102015D2331A721
:10AB000010D00601915102015A5F060192510201D3
:10AB10005B5B0601935102015C5B060194510201EB
:10AB20005D5B07A523D0EE0EF66E170EF76E150EC1
:10AB30000A01E16F0001B1EC0CF0080EE96EF0C6FD
:10AB4000E4FAEFC6E3FAEEC6E2FAEDC6E1FA3FEC4C
:10AB500020F0200E9EA8FED7AD6E0A0E9EA8FED74E
:10AB6000AD6E0D0E9EA8FED7AD6E020107A522D0D8
:10AB70000C0EF66E180EF76E140E0A01E16F00014E
:10AB8000B1EC0CF0080EE96E5DC2E4FA5CC2E3FAC7
:10AB90005BC2E2FA5AC2E1FA3FEC20F0200E9EA816
:10ABA000FED7AD6E0A0E9EA8FED7AD6E0D0E9EA806
:10ABB000FED7AD6E0601FD5318E1D8900201526B2D
:10ABC0005A35536F5B35546F5C35556F276B266B69
:10ABD000020E256F246BC8C661F2C7C660F2C6C6F6
:10ABE0005FF2C5C65EF219D00601FD2D16D05DC21A
:10ABF00055F25CC254F25BC253F25AC252F20201E5
:10AC0000276B266B256B010E246F94C661F293C6E9
:10AC100060F292C65FF291C65EF2020107A52FD0E4
:10AC2000280EF66E180EF76E0D0E0A01E16F000188
:10AC3000B1EC0CF055C2E1FA570E0A01E26F0001C7
:10AC4000C6EC0CF054C2E1FA570E0A01E26F0001A3
:10AC5000C6EC0CF053C2E1FA570E0A01E26F000194
:10AC6000C6EC0CF052C2E1FA570E0A01E26F000185
:10AC7000C6EC0CF0200E9EA8FED7AD6E020155C2A8
:10AC80003DF254C23CF253C23BF252C23AF25E5120
:10AC90005225006E5F515321016E60515421026EA6
:10ACA00061515521036E00503A5D0AE101503B5D50
:10ACB00007E102503C5D04E103503D5DD8B492D100
:10ACC00080A023D0010E1C27D8B01D2BD8B41E2B7A
:10ACD000D8B41F2B17511F5D11E30BE116511E5DF8
:10ACE0000DE307E115511D5D09E303E11C51145DFE
:10ACF00005E21F6B1E6B1D6B010E1C6F00011BEC30
:10AD00004CF067EF52F048D0020183AC1FD0FF0E29
:10AD10001C27D8A01D27D8A01E27D8A01F271C534A
:10AD20000EE11D530CE11E530AE11F5308E117C247
:10AD30001FF216C21EF215C21DF214C21CF200014F
:10AD40001BEC4CF067EF52F027D0020180A212D02A
:10AD5000375110080FE23707020E0801526F0B0E31
:10AD6000536F37C254F837C255F8000181EC0CF02C
:10AD700013D0020183AE11D0373D01D00ED0372B56
:10AD8000020E0801526F0B0E536F37C254F837C2D0
:10AD900055F8000181EC0CF00201596B586B576BB0
:10ADA000566B356B346B336B326B0101BE51BD5D3D
:10ADB0000CE00001ABEC4EF0012C04D01BEC4CF08D
:10ADC00067EF52F00201F1D7010180A44FD0010ECC
:10ADD00002015627D8B0572BD8B4582BD8B4592BCA
:10ADE000010E0801456F00017AEC11F0020107B372
:10ADF0003BD0595307E1585305E1575303E15651EE
:10AE0000F90832E20A01DE6B300EDF6F0001C2EC9E
:10AE10000EF0020E0201876F866F856B846B0F0E3A
:10AE2000836FFF0E826F3A0EF66E180EF76E0001FA
:10AE30006AEC11F0020107810793020E0801526FBC
:10AE4000070E536F1E0E546F040E556F000181ECF8
:10AE50000CF0020E0801526F060E536F546B030E76
:10AE6000556F000181EC0CF00101AFD7020107B36F
:10AE70003BD0565306E1575304E1585302E159536E
:10AE800033E0595331E158532FE157532DE15651D7
:10AE9000F9082AE3078336C871F235C870F234C85E
:10AEA0006FF233C86EF20A01DE6B300EDF6F000105
:10AEB000C2EC0EF0020E0201876F866F0801446F2C
:10AEC000000146EC3BF05FEC4CF0140E0801456FBE
:10AED00000017AEC11F00201596B586B576B566BFD
:10AEE000010173D76AD0020107A333D0565306E19C
:10AEF000575304E1585302E159532BE007930A01D9
:10AF0000DE6B300EDF6F0001C2EC0EF0020E0201AC
:10AF1000876F866F030E0801446F000146EC3BF01B
:10AF2000020E0801526F070E536F1E0E546F040E6F
:10AF3000556F000181EC0CF0020E0801526F060EF5
:10AF4000536F546B010E556F000181EC0CF035D03E
:10AF5000020107A332D080B41BD083BC19D080B0CB
:10AF600017D080B215D083BE13D000019FEC3DF006
:10AF70000101BE51BD5D0AE00001ABEC4EF0015095
:10AF8000020803E1010121D70001F2D70201E3D752
:10AF900080A403D008B101D000D783AC0DD008B194
:10AFA0000BD000011BEC4CF089EC0EF00C0E0201F2
:10AFB000106F08852DD001D0CED73DC247F83CC2D6
:10AFC00046F83BC245F83AC244F800016DEF51F033
:10AFD000020124513A2725513B2326513C23275176
:10AFE0003D2355D631B909D0F4C6F0F6F3C6EFF6D5
:10AFF000F2C6EEF6F1C6EDF607D031A905D0000194
:10B000001BEC4CF0020104D000011AD5080102012A
:10B01000000114EF58F0020110510A082FE100015D
:10B020009FEC3DF067EF52F00201135309E100017C
:10B0300089EC0EF00B0E0201106F08953195ECD7DC
:10B0400012531CE1010E1C27D8B01D2BD8B41E2BA7
:10B05000D8B41F2B17511F5D11E30BE116511E5D74
:10B060000DE307E115511D5D09E303E11C51145D7A
:10B0700005E21F6B1E6B1D6B010E1C6F10510B0840
:10B08000D8A40AD1010E876F866F088383AC08D0DD
:10B09000FA0E0801456F00017AEC11F00201F6D7B3
:10B0A00000019FEC3DF00201356B346B336B326B6A
:10B0B00080B42AD083BC28D080B026D080B224D0DF
:10B0C00083BE22D00101BE51BD5D1FE00001ABEC8B
:10B0D0004EF0012C17D00A0E0201106F030E08016A
:10B0E000446F000195EC2AF0020E0801446F000144
:10B0F00095EC2AF002011F6B1E6B06C21DF205C201
:10B100001CF204D30201DED70101020108A327D0FB
:10B11000286B000189EC0EF00201856B0F0E846F25
:10B12000836FFF0E826F0A01DE6B380EDF6F000146
:10B13000C2EC0EF01C0EF66E150EF76E6AEC11F0F6
:10B14000030E0801446F000195EC2AF02E0EF66EF6
:10B15000150EF76E2FEC0CF002010881089383AEF8
:10B160002CD008810F510D5D02E20D2B05D00F513F
:10B170000D5D02E1010E0D6F3E0EF66E150EF76EBF
:10B18000130E0A01E16F0001B1EC0CF00DC2E1FAFF
:10B19000570E0A01E26F0001C6EC0CF0200E9EA8CB
:10B1A000FED7AD6E0A0E9EA8FED7AD6E0D0E9EA800
:10B1B000FED7AD6E020108832BD080A229D0088172
:10B1C0000D510008D8A00D070D5302E10FC20DF27A
:10B1D000580EF66E150EF76E130E0A01E16F0001A0
:10B1E000B1EC0CF00DC2E1FA570E0A01E26F00015A
:10B1F000C6EC0CF0200E9EA8FED7AD6E0A0E9EA8DF
:10B20000FED7AD6E0D0E9EA8FED7AD6E020108836F
:10B2100080A041D008A13FD0000189EC0EF0036A64
:10B2200002010D51FE0FE96E060E0320EA6EEF508B
:10B23000000803E20C0E106F2DD0036A0D51FE0FB3
:10B24000E96E060E0320EA6EEF5224E10A01DE6B7E
:10B25000180EDF6F0001C2EC0EF0010E0201876FC5
:10B26000866F856B846B0F0E836FF00E826F720E8C
:10B27000F66E150EF76E00016AEC11F0020E080171
:10B28000446FFA0E456F00017AEC11F00801442F6B
:10B29000F8D70201C1D60CD710510C08D8A436D269
:10B2A000010E876F866F00019FEC3DF00201089749
:10B2B000020E0801446F000195EC2AF01FC223F230
:10B2C0001EC222F21DC221F21CC220F2820EF66EB4
:10B2D000150EF76E140E0A01E16F0001B1EC0CF0CF
:10B2E000410EE96E23C2E4FA22C2E3FA21C2E2FA75
:10B2F00020C2E1FA3FEC20F0990EF66E150EF76EC3
:10B300000B0E0A01E16F0001B1EC0CF0020108879D
:10B310000885089131B50897356B346B336B326B08
:10B3200080B409D083BC07D080B005D080B203D0F0
:10B3300083BE01D00BD083AC09D0000189EC0EF0A4
:10B340000B0E0201106F0895319566D608A727D01D
:10B35000296B000189EC0EF00F0E0201856FF00ED3
:10B36000846F836B826B0A01DE6B380EDF6F000126
:10B37000C2EC0EF0A60EF66E150EF76E6AEC11F02A
:10B38000010E0801446F000195EC2AF0B80EF66E2C
:10B39000150EF76E2FEC0CF002010885089783AEAE
:10B3A000A1D00885036A0D51FE0FE96E060E032039
:10B3B000EA6EEF5020250801446F000E02012121A2
:10B3C0000801456F000E020122210801466F000EA0
:10B3D000020123210801476F010E445D006E000E3B
:10B3E0004559016E000E4659026E000E4759036E14
:10B3F00002011F51035C15E30BE11E51025C11E3D6
:10B4000007E11D51015C0DE303E100501C5D09E201
:10B41000010E1C27D8B01D2BD8B41E2BD8B41F2B5F
:10B420003BD0036A0D51FE0FE96E060E0320EA6E53
:10B43000EF5020250801446F000E02012121080170
:10B44000456F000E020122210801466F000E020125
:10B4500023210801476F010E445D006E000E45591F
:10B46000016E000E4659026E000E4759036E0050E1
:10B4700002011C5D11E101501D5D0EE102501E5DD7
:10B480000BE103501F5D08E123C21FF222C21EF22E
:10B4900021C21DF220C21CF2C80EF66E150EF76E08
:10B4A000140E0A01E16F0001B1EC0CF0410EE96EDF
:10B4B0001FC2E4FA1EC2E3FA1DC2E2FA1CC2E1FA9C
:10B4C0003FEC20F0200E9EA8FED7AD6E0A0E9EA87F
:10B4D000FED7AD6E0D0E9EA8FED7AD6E0201088799
:10B4E000319579D080A277D0088523511F5D15E36F
:10B4F0000BE122511E5D11E307E121511D5D0DE3BA
:10B5000003E11C51205D09E2FF0E1C27D8A01D2776
:10B51000D8A01E27D8A01F2739D020511C5D36E1A6
:10B5200021511D5D33E122511E5D30E123511F5D2C
:10B530002DE1036A0D51FE0FE96E060E0320EA6E3F
:10B54000EF5020250801446F000E0201212108015F
:10B55000456F000E020122210801466F000E020114
:10B5600023210801476F010E445D02011C6F000E8C
:10B570000801455902011D6F000E080146590201DC
:10B580001E6F000E0801475902011F6FE40EF66E90
:10B59000150EF76E140E0A01E16F0001B1EC0CF00C
:10B5A000410EE96E1FC2E4FA1EC2E3FA1DC2E2FABE
:10B5B0001CC2E1FA3FEC20F0200E9EA8FED7AD6E33
:10B5C0000A0E9EA8FED7AD6E0D0E9EA8FED7AD6EDC
:10B5D00002010887319580B002D080A496D008A5DA
:10B5E00094D03195000EF66E160EF76E140E0A0109
:10B5F000E16F0001B1EC0CF0410EE96E23C2E4FAF8
:10B6000022C2E3FA21C2E2FA20C2E1FA3FEC20F0C2
:10B61000170EF66E160EF76E090E0A01E16F0001A5
:10B62000B1EC0CF0220EF66E160EF76E120E0A0139
:10B63000E16F0001B1EC0CF0410EE96E1FC2E4FABB
:10B640001EC2E3FA1DC2E2FA1CC2E1FA3FEC20F08E
:10B65000370EF66E160EF76E090E0A01E16F000145
:10B66000B1EC0CF0420EF66E160EF76E0D0E0A01DE
:10B67000E16F0001B1EC0CF029C2E1FA1B0E0A01E6
:10B68000E26F0001B5EC20F0510EF66E160EF76E6B
:10B69000090E0A01E16F0001B1EC0CF0036A02012E
:10B6A0000D51FE0FE96E060E0320EA6EEFCF44F84F
:10B6B0005C0EF66E160EF76E1C0E0A01E16F0001AD
:10B6C000B1EC0CF044C8E1FA1B0E0A01E26F000174
:10B6D000B5EC20F07A0EF66E160EF76E0D0E0A011E
:10B6E000E16F0001B1EC0CF0020108BB0ED0036A5F
:10B6F0000D51FE0FE96E060E0320EA6EEF5205E0D3
:10B700000A0E106F0895089187D40AD60001A1EFA0
:10B710005CF0F86AD09E078E5E0E006E100E016E11
:10B72000020EE96E000EEA6EEE6A002EFDD7012EC3
:10B73000FBD7EA6AE96A700ED36E400E9B6ED35057
:10B74000B8868A0EAF6E000EB06EA60EAC6E900E6E
:10B75000AB6E0101BD6BBE6B000E7E6EC198C19ACF
:10B760007F50E00B7F6E799A79987A6A7B6A196AC2
:10B770001A6A700ED36E400E9B6ED350080E7E6E0A
:10B78000C198C19A7F50E00B7F6EC050C00B060974
:10B79000C06EC08EC2800F0E926E0B0E936E800E26
:10B7A000946ED10E956E9690968296849686C00E73
:10B7B000F2129D8A0F0E0201386FFF0E396FF2CF21
:10B7C00043F8F29EAA6A010EA96EA69CA69EA680C8
:10B7D000A850080143BFF28E0201376F373D02D0F7
:10B7E000400E376FF2CF43F8F29EAA6A020EA96E9E
:10B7F000A69CA69EA680A850080143BFF28E020117
:10B80000126F123D01D0126BF2CF43F8F29EAA6A7A
:10B81000030EA96EA69CA69EA680A850080143BF51
:10B82000F28E0201136F133D02D0010E136F8B8A4B
:10B83000899E9E0EF66E140EF76E00012FEC0CF032
:10B84000A40EF66E140EF76E2FEC0CF0D00EF66E02
:10B85000140EF76E2FEC0CF0E9EF0CF0E20EF66E22
:10B86000140EF76E2FEC0CF0BAEF0DF089EC0EF021
:10B87000060E0A01DE6F080EDF6F0001C2EC0EF04B
:10B88000020E0201876F866F0F0E856F846B836FC8
:10B89000FF0E826FF40EF66E140EF76E00016AEC66
:10B8A00011F0120E0A01DE6F180EDF6F0001C2ECFC
:10B8B0000EF0020E0201876F010E866F856B846B9E
:10B8C000836BF00E826FFE0EF66E140EF76E0001A3
:10B8D0006AEC11F00A01DE6B300EDF6F0001C2EC82
:10B8E0000EF0010E0201876F866F856B846B0F0E61
:10B8F000836FF00E826F0A0EF66E150EF76E000162
:10B900006AEC11F00201079508998D900001AFECE7
:10B910003CF0020108A905D00001AFEC3CF0F9D7DA
:10B92000020108B904D0000159EC3AF0020131815A
:10B9300031936D6B6C6B6B6B010E6A6F00010BEFDB
:06B9400058F0FDD70300E2
:020000040030CA
:0E00000000C8181E008F80000FC00FE00F40D8
:00000001FF
